:1000000000400020354D0000754D0000774D000088
:1000100000000000000000000000000000000000E0
:10002000000000000000000000000000794D00000A
:1000300000000000000000007B4D00007D4D00002E
:100040007F4D0000DD2C0000695500007F4D000051
:100050007F4D0000000000007F4D00007F4D00003C
:100060007F4D0000AD4F00007F4D00007F4D000030
:100070007F4D00007F4D00007F4D00007F4D000050
:100080007F4D00000D5600007F4D00007F4D0000A9
:100090007F4D00007F4D00007F4D00007F4D000030
:1000A0007F4D00007F4D00000000000000000000B8
:1000B0000000000000000000000000000000000040
:1000C000054B0648033310B51B1A062B03D9044B06
:1000D000002B00D0984710BD2002002020020020F5
:1000E000000000000648074910B5091A8910CB0F17
:1000F0005918491003D0044B002B00D0984710BD6D
:1001000020020020200200200000000010B5074C53
:100110002378002B09D1FFF7D3FF054B002B02D02A
:10012000044800E000BF0123237010BD200200201E
:1001300000000000F08A0000094B10B5002B03D02E
:100140000849094800E000BF08480368002B02D1B5
:10015000FFF7C8FF10BD064B002BF9D09847F7E713
:100160000000000024020020F08A00001C02002091
:1001700000000000164B002B00D1144B9D4640227E
:1001800092029A1A924600218B460F461348144A4F
:10019000121A06F07EFB0F4B002B00D098470E4B37
:1001A000002B00D098470020002104000D000D48CE
:1001B000002802D00C4800E000BF06F027FB20001A
:1001C000290005F0E9F906F0FBFAC0460000080036
:1001D000004000200000000000000000200200207D
:1001E000D024002000000000000000000123034094
:1001F0000200181E04D1042A03D91068000900E087
:100200000020704710B50400FFF7F0FF0300002046
:1002100083420BD0013B9B00181DE2181279002A83
:1002200003D001338342F8D100E0180010BD012251
:10023000016810B5114201D0002903DA102000F046
:10024000E3F903E04910062001F004FF10BD016846
:1002500010B5CB0701D5002903DA102000F0D4F93E
:1002600006E04910033189100022052001F0F2FE5A
:1002700010BD70B50568AB0728D1042D26D90F2312
:100280002A6846681340062B09D12800FFF7AEFF05
:10029000012383421DDC9A00AE500133F9E7052BA0
:1002A00014D1F30703D4132000F0AEF912E0761056
:1002B000FF2EF8D82800FFF799FF2C1D230080009F
:1002C0002018984205D91E700133FAE70B2000F080
:1002D0009BF9002070BD70B50468E30701D41120BC
:1002E0002DE04568AB0729D1042D27D90F262B68AF
:1002F00064101E40062E0BD1002C04DD2800FFF7F1
:1003000075FF844201DD122019E0A400605918E055
:10031000331F012B12D82800FFF768FF8000042E3E
:1003200002D12800FFF76EFF002CECDDA042EADBD3
:1003300001232C19E0784000184302E00B2000F064
:1003400063F970BDF8B5012304681C4201D1112086
:100350002FE00325466835402AD1042E28D90F23E3
:100360003268641087681340062B0BD1002C04DD23
:100370003000FFF73BFF844201DD122019E0A400AA
:10038000A75113E0052B13D1002CF6DD3000FFF749
:100390002DFF80008442F0DC01231F4201D1132095
:1003A00007E07F10FF2FFAD83419E770280002E029
:1003B0000B2000F029F9F8BD006810B5830717D1AC
:1003C000042815D90F2302681340062B02D1FFF72A
:1003D0000DFF0BE0052B05D1FFF708FFC00001233F
:1003E000184308E0042B03D1FFF70CFF4000F6E7A9
:1003F0000B2000F009F910BD10B50324006804407B
:1004000006D1042804D90F2302681340042B01D01D
:100410000E2011E001F05AFE0378233B5942594166
:1004200010224018210006F00DFF80239B05C21802
:10043000054B9A4203D9142000F0E6F802E00123AC
:100440004000184310BDC046FFFFFF3F10B5012418
:100450000368234202D04268224203D10D2000F0FB
:10046000D3F808E004495B1052101B070A401343FD
:1004700018684000204310BDFCFFFF0F01210368F6
:1004800010B50B4205D042680A4202D0806808428B
:1004900003D10D2000F0B8F808E005495B105210B8
:1004A0001B070A40401013431860002010BDC046CF
:1004B000FCFFFF0F012303400200181E01D0501063
:1004C00002E00D22014B1A707047C0463C0200202A
:1004D000012303400200181E04D1042A03D9106826
:1004E000000900E00020704770B50D000400FFF720
:1004F000EFFF86002800FFF7EBFF830000209E42FD
:100500000ED1231D9E1904351A009E4207D9297861
:100510001278013301358A42F6D0002000E0012034
:1005200070BD0000F0B585B00393019002912D4E8F
:100530002D4B002A02D002223270013A00251A60A7
:100540001B68F554019B9D424ADA029AAB00D058D1
:10055000254B1C68C8239B0037191C1B012318421C
:1005600002D04310214A1FE0214A002802D004286B
:1005700005D1204A2100380006F052FD18E0042879
:1005800010D90F2302681340042B04D101F09EFD03
:10059000194A030008E0062B05D1FFF799FF174A17
:1005A000030001E00123164A2100380006F038FD5F
:1005B000300006F09BFD039B0B4A002B01D110601D
:1005C0000CE0019B013B9D42F9DA0E4B9842F6DCB0
:1005D000431C1360202232540022F2540135B1E74B
:1005E00005B0F0BD48020020440200201180000048
:1005F000E47F0000EA7F000039830000EF7F000005
:10060000008000001F030000014B1870002070479D
:100610003C02002070B503F0B7F9094C0100251D1C
:100620001F22280006F069FD280006F05FFD042364
:1006300004308008000118432060200070BDC046CF
:1006400068050020C368F0B59D00836887B05D1918
:10065000030018330393036902909F00039BDF1983
:1006600043699E000093039B9E19D24B1B78002B7D
:100670000FD17F222B68D0491C1213409B005B587E
:1006800000960435019235E0CA4B1B78002B29D027
:10069000009E029BC74C9B6821780093EA1A029B3C
:1006A00092109B7812021A43029B587802F0F8FECF
:1006B0000023029A2370137000960497029B039AFA
:1006C0009B68ED1A0193029BAD10DD60049B9F1A9D
:1006D000029BBF101F61009B9B1A029A9B105361E3
:1006E00001F005FC2B68019A1C121340B24A9B00D2
:1006F0009B5804359F46029B587802F0C9FE0023A0
:10070000029A1370D9E7039B3A1DD11AA94BDB2932
:1007100003DD1A22009E1A70BBE71B783C60002B99
:1007200002D0009E1700B4E72B6801991C120B4001
:10073000A1499B005B5817000435DBE7039B3A1D7A
:10074000D11A9C4BDB2903DD1A22009E1A70A0E708
:1007500028681B78291D3860002B03D0009E1700E5
:100760000D0096E76B6801991C120B4092499B00A3
:100770005B5817000835BDE7039B3A1DD11A8D4B16
:10078000DB2903DD1A22009E1A7082E7A4001B7881
:100790002C193C60002B02D0009E170079E72B68D3
:1007A00001991C120B4084499B005B5817000435CB
:1007B000A0E7039B3A1DD11A7E4BDB2903DD1A22E9
:1007C000009E1A7065E77D48A40021581B783960A7
:1007D000002B02D0009E17005BE72B6801991C12CA
:1007E0000B4075499B005B581700043582E7043FB6
:1007F000724B3A68A400E2506E4B1B78002B01D07C
:10080000009E46E72B68019A1C1213406A4A9B001F
:100810009B5804356EE7694BA600F058FFF74AFE77
:10082000043F04003868FFF745FE24180120634B9D
:1008300064000443F4505F4B1B78002B01D0009EF2
:1008400027E72B68019A1C1213405B4A9B009B58B8
:1008500004354FE7039B3A1DD11A564BDB2903DDC4
:100860001A22009E1A7014E70098039C0121A042EE
:1008700002D901000C3909681B783960002B02D0BD
:10088000009E170005E72B6801991C120B404A498E
:100890009B005B58170004352CE7039B3A1DD11AC7
:1008A000444BDB2903DD1A22009E1A70F1E6009901
:1008B000039881420AD90B000C3B1B6840495B102E
:1008C0006418E41A009BA400E35802E01821197090
:1008D00000233B60374B1B78002B02D0009E170093
:1008E000D7E62B6801991C120B4033499B005B58DB
:1008F00017000435FEE6009B039A93420BD90C3B8C
:1009000019682F4B043FE3184910591A3A68009BA5
:100910008900CA5002E01822264B1A70254B1B781A
:10092000002B01D0009EB4E62B68019A1C121340E4
:10093000214A9B009B580435DCE6009B039A9342B6
:100940001CD9009E1E4B0C3EE4183368009A5B10C5
:10095000E31A9B009858FFF7ADFD043F04903868F8
:10096000FFF7A8FD3168049B4910611A012418188B
:100970004000009B89002043C85002E018220D4B24
:100980001A700C4B1B78002B01D0009E81E62B685F
:10099000019A1C121340084A9B009B580435A9E693
:1009A000039B3A1DD11A034BDB290BDD1A22009E53
:1009B0001A706EE63C020020E47D0000382300201F
:1009C000FDFFFF3F0099A40061581B783960002BA0
:1009D00002D0009E17005CE62B6801991C120B40A8
:1009E000CF499B005B581700043583E6043F009B0A
:1009F0003A68A400E250CB4B1B78002B01D0009E3C
:100A000047E62B68019A1C121340C54A9B009B586D
:100A100004356FE6009BA4001C192368043F386866
:100A20005E10FFF747FD36180120BE4B76001B789D
:100A300006432660002B01D0009E2AE62B68019A0F
:100A40001C121340B64A9B009B58043552E6039B88
:100A5000A4003F1BB34CBB420DD82378002B01D020
:100A6000009E16E62B68019A1C121340AC4A9B00AC
:100A70009B5804353EE6AC4801F09EFA2378002BE3
:100A800001D0009E05E62B68019A1C121340A44A6F
:100A90009B009B5804352DE6A300ED18002C00DACE
:100AA0000BE6A04B1B78002B01D0009EF1E52B68D4
:100AB000019A1C1213409A4A9B009B58043519E670
:100AC0003B1F04931B680593042B04D1A300ED186E
:100AD000002C00DAF2E5934B1B78002B02D0009E2D
:100AE000049FD6E52B68019A1C1213408C4A9B0088
:100AF0009B58049F0435FDE53B1F04931B68059339
:100B0000002B04D1A300ED18002C00DAD6E5854BAC
:100B10001B78002B02D0009E049FBAE52B68019A37
:100B20001C1213407E4A9B009B58049F0435E1E54C
:100B30003A1F13685B10013B002B07DD01215B00AE
:100B4000A4000B4304972D191360B7E5754B1700EC
:100B50001B78002B01D0009E9BE52B68019A1C128C
:100B600013406F4A9B009B580435C3E53A00039B32
:100B70000C32D31ADB2B04DD1A226A4B009E1A704A
:100B800087E5FF2361005B000B4001210B433B60C5
:100B9000029B03989B6824120493ED1A029BAD10EC
:100BA0009B782D021D43009B8D401B1A9B108B4090
:100BB0000B43BB60029B0D437D609C70E4B25B4BBA
:100BC000E4000299E35816008B6056490978002921
:100BD00003D008331D0017005BE51D0001999B68D9
:100BE0000C351C120B404E499B005B5800921700BD
:100BF00080E53B1F1E68039A009B93422AD104970D
:100C00000A20F30716D4B3070DD1042E0BD90F23F6
:100C100032681340042B06D1300001F057FA06F079
:100C200065FA063006E00720042E03D0002E01D01E
:100C300080208000643002F0DBF9002801D1043DFF
:100C40003CE5029B3100587802F03CFC0023029AFC
:100C5000137033E5009B009A0C3B1B6802995B10F4
:100C60009B005B421F00D3180C3B1E601300083B27
:100C70001B68083FD7195A108A70D2B22B49D2008C
:100C80005B0055589B0A029A9B009560ED18009BEB
:100C9000043B1E68039B7610B6009E19214B1B78FF
:100CA000002B00D0F5E42B68019A1C1213401C4A5B
:100CB0009B009B58009604351CE53B1F1868FFF706
:100CC000F9FBA40006003F1B1E2833DC00280EDCC5
:100CD000144B1B78002B01D0009EDAE42B68019A9C
:100CE0001C1213400E4A9B009B58043502E502F08B
:100CF00031FE033E361802F02DFE0D4B801B98424C
:100D0000F9D8084B1B78002B01D0009EC1E42B685A
:100D1000019A1C121340024A9B009B580435E9E4D7
:100D2000E47D00003C02002014800000401B0020F5
:100D30009F8601000123029A137002F00BFE029BB2
:100D40000A3886195E60B8E43B1F1868FFF7B2FBEB
:100D5000A40004903F1B00280EDCCF4B1B78002B17
:100D600001D0009E95E42B68019A1C121340CB4AD7
:100D70009B009B580435BDE4C94B049A009E9A42DF
:100D800003DD1D22C44B1A7083E40123029A137001
:100D900002F0E0FDFA23049A9B005343029A0A3BB7
:100DA0001B18536089E4A300FF1A002320001A00D7
:100DB0003900FFF7B7FBBB4EBB4C3168200002F097
:100DC000CDFA3168200002F084FBB34B1B78002B76
:100DD00001D0009E5DE42B68019A1C121340AF4ABB
:100DE0009B009B58043585E4AB4BA4001B783F1B4C
:100DF000002B01D0009E4CE42B68019A1C1213407A
:100E0000A64A9B009B58043574E402F037F901F0C0
:100E10006EF83B1F1868002823D1083B1868C307E9
:100E200001D5401016E083070FD104280DD90F23F8
:100E300002681340062B02D1FFF74AFB0AE0052B9C
:100E400003D1FFF745FB800004E01922924B009E7E
:100E50001A701EE43A0001214300083A0B43136064
:100E600001E040100138002832DD01224300134325
:100E7000391F0B603B00083B1B681341181A3B00ED
:100E80000C3B1B68134203D08018A400904015E06F
:100E9000990717D1042B15D90F211E683140062957
:100EA00006D101308000C358009AA400A35010E07E
:100EB000052907D118180079A4004000009B1043B1
:100EC000E05006E01922744B009E1A70FFF7E1FB18
:100ED0000435714B1B78002B02D0009EFFF7D9FB25
:100EE0002B68019A1C1213406C4A9B009B580435D6
:100EF000FFF700FCA300039AFB189B1ADB2B01DC15
:100F0000002205E01A22644B009E1A70FFF7C1FB15
:100F1000631E002C03DD3A601C000437F8E75E4BCB
:100F20001B78002B02D0009EFFF7B3FB2B68019AC1
:100F30001C121340594A9B009B580435FFF7DAFBFB
:100F4000A3009C46F81A002C04DC1C22524B0026FD
:100F50001A7015E0002103685B1001268A00825890
:100F6000164003D10D224C4B1A7009E052109342E7
:100F700000DD130001318C42EFDC01265B001E43D3
:100F80006346FF1A444B06601B780437002B02D0DF
:100F9000009EFFF77EFB2B68019A1C1213403F4A0C
:100FA0009B009B580435FFF7A5FBA3009C46F81A4D
:100FB000002C04DC1C22384B00261A7015E000219E
:100FC00003685B1001268A008258164003D10D2267
:100FD000314B1A7009E05210934200DA13000131CC
:100FE0008C42EFDC01265B001E436346FF1A2A4B4E
:100FF00006601B780437002B02D0009EFFF749FBE8
:101000002B68019A1C121340244A9B009B580435FC
:10101000FFF770FB3B00083B1868FFF74BFA3B1FDC
:1010200004901868FFF746FA049AA600BC1B002338
:10103000824200DA04332360174BBF1B1B7804374E
:10104000002B02D0009EFFF724FB2B68019A1C1294
:101050001340124A9B009B580435FFF74BFBA3003B
:10106000FE1A04933B00083B1868FFF723FA3B1F66
:1010700004001868FFF71EFAE20FC317A04253419D
:101080009B003360049BFF1A034B04371B78002B33
:101090000CD0009EFFF7FDFA3C020020E47D00002A
:1010A00080EE360044020020480200202B68019A9E
:1010B0001C121340D84A9B009B580435FFF71AFBBB
:1010C0003B00083B18683B1F1968A300884202D107
:1010D000FB1A042222E004281ED90122104201D06A
:1010E000114219D10326304215D10F2302681A404C
:1010F000042A10D131420ED104290CD90A681340B8
:10110000042B08D1FFF7F0F9431E9841A600BE1B3F
:101110008000306003E0A3000022FB1A1A60BF4B7E
:10112000A4001B783F1B0437002B02D0009EFFF762
:10113000B0FA2B68019A1C121340B74A9B009B58C7
:101140000435FFF7D7FA3B00083B18683B1F1968C6
:10115000A300884202D1FB1A002223E004281FD9F1
:101160000122104201D011421AD10326304216D179
:101170000F2302681A40042A11D131420FD10429E9
:101180000DD90A681340042B09D1FFF7ADF903000C
:1011900058425841A600BE1B8000306003E0A30007
:1011A0000422FB1A1A609D4BA4001B783F1B0437D6
:1011B000002B02D0009EFFF76CFA2B68019A1C12DC
:1011C0001340954A9B009B580435FFF793FAA30000
:1011D000FE1A04933B00083B1868FFF76BF93B1FAE
:1011E00004001868FFF766F9E217C30F8442534101
:1011F0009B003360049BFF1A884B04371B78002B3D
:1012000002D0009EFFF745FA2B68019A1C1213408A
:10121000814A9B009B580435FFF76CFA3B00083B62
:101220001868FFF747F93B1F04901868FFF742F969
:10123000049AA600BC1B0023824200DD0433236015
:10124000764BBF1B1B780437002B02D0009EFFF7A4
:1012500020FA2B68019A1C1213406F4A9B009B587E
:101260000435FFF747FA3B1F1B686C4AA400042BA8
:1012700002D13B1B002103E0002B03D104213B1BC7
:10128000196001E00C23137013783F1B0437002B07
:1012900002D0009EFFF7FDF92B68019A1C12134043
:1012A0005D4A9B009B580435FFF724FAA300FC1A03
:1012B00004933B00083B1868FFF7FCF83B1F06004F
:1012C0001868FFF7F7F836180120049B7600FF1A1C
:1012D000524B06431B7826600437002B02D0009E39
:1012E000FFF7D7F92B68019A1C1213404A4A9B005A
:1012F0009B580435FFF7FEF9A300FE1A04933B0048
:10130000083B1868FFF7D6F83B1F04001868FFF782
:10131000D1F8241A0120049B6400FF1A3F4B0443B8
:101320001B7834600437002B02D0009EFFF7B1F920
:101330002B68019A1C121340374A9B009B580435B6
:10134000FFF7D8F9A300FC1A04933B00083B186888
:10135000FFF7B0F83B1F06001868FFF7ABF84643ED
:101360000120049B7600FF1A2C4B06431B78266055
:101370000437002B02D0009EFFF78BF92B68019AEF
:101380001C121340244A9B009B580435FFF7B2F906
:101390003B00083B1868FFF78DF83B1F0490186866
:1013A000FFF788F80100049804F0FEF90123A40077
:1013B0003E1B370040001843184B30601B78043741
:1013C000002B02D0009EFFF764F92B68019A1C12D3
:1013D0001340114A9B009B580435FFF78BF93B00E3
:1013E000083B1868FFF766F83B1F04901868FFF782
:1013F00061F80100049804F0BDFA0123A4003E1B2B
:10140000370049001943054B31601B780437002B26
:1014100006D0009EFFF73DF9E47D00003C0200206D
:101420002B68019A1C121340E74A9B009B58043515
:10143000FFF760F93B1F1868FFF73CF8C317C018A7
:101440005840012340001843E04BA4001B783E1B8A
:101450003060371D002B02D0009EFFF71AF92B6871
:10146000019A1C121340D84A9B009B580435FFF781
:1014700041F9A300FE1A05933068012C03D1FFF750
:1014800019F8049008E0FFF715F804007068FFF7FA
:1014900011F80130031B0493049B002B01DC012392
:1014A000049305F06FFD049904F064FA0C1901210E
:1014B000059B6400FF1AC54B0C431B78346004374E
:1014C000002B02D0009EFFF7E4F82B68019A1C1253
:1014D0001340BD4A9B009B580435FFF70BF9A4004D
:1014E0003E1B3000FEF788FFB84B30601B78371D7D
:1014F000002B02D0009EFFF7CCF82B68019A1C123B
:101500001340B14A9B009B580435FFF7F3F8A30042
:10151000FE1A04933B00083B1868FEF7CBFF3B1F05
:1015200004001868FEF7C6FF04400120049B640015
:10153000FF1AA64B04431B7834600437002B02D0FB
:10154000009EFFF7A6F82B68019A1C1213409E4AD2
:101550009B009B580435FFF7CDF8A300FC1A0493B9
:101560003B00083B1868FEF7A5FF3B1F0600186804
:10157000FEF7A0FF06430120049B7600FF1A934B61
:1015800006431B7826600437002B02D0009EFFF72D
:1015900080F82B68019A1C1213408B4A9B009B58C1
:1015A0000435FFF7A7F8A300FC1A04933B00083B9F
:1015B0001868FEF77FFF3B1F06001868FEF77AFFEA
:1015C00046400120049B7600FF1A804B06431B789F
:1015D00026600437002B02D0009EFFF75AF82B68D4
:1015E000019A1C121340784A9B009B580435FFF760
:1015F00081F83B1F1868FEF75DFFC04301234000E0
:101600001843724BA4001B783E1B3060371D002B23
:1016100002D0009EFFF73DF82B68019A1C12134080
:10162000694A9B009B580435FFF764F8A300FE1A33
:1016300004933B00083B1868FEF73CFF3B1F040087
:101640001868FEF737FF8440012364001C43049BA5
:101650003460FF1A5D4B04371B78002B02D0009ECC
:10166000FFF717F82B68019A1C121340564A9B008B
:101670009B580435FFF73EF8A300FE1A04933B0085
:10168000083B1868FEF716FF3B1F04001868FEF7BA
:1016900011FF0441012364001C43049B3460FF1AC2
:1016A0004A4B04371B78002B02D0009EFEF7F1FF57
:1016B0002B68019A1C121340434A9B009B58043527
:1016C000FFF718F8A4003E1B3000FEF7B0FD3F4BBB
:1016D00030601B78371D002B02D0009EFEF7D9FF2B
:1016E0002B68019A1C121340374A9B009B58043503
:1016F000FFF700F8A4003E1B3000FEF7A8FD334BB7
:1017000030601B78371D002B02D0009EFEF7C1FF12
:101710002B68019A1C1213402B4A9B009B580435DE
:10172000FEF7E8FFA4003F1B3800FEF7A2FD274BA1
:101730001B78002B02D0009EFEF7ABFF2B68019AAE
:101740001C121340204A9B009B580435FEF7D2FF21
:10175000A4003E1B3000FEF7BEFD1C4B30601B7822
:10176000371D002B02D0009EFEF793FF2B68019AD5
:101770001C121340144A9B009B580435FEF7BAFF15
:10178000A4003F1B3800FEF7DDFD104B1B78002B3B
:1017900002D0009EFEF77DFF2B68019A1C121340B9
:1017A000094A9B009B580435FEF7A4FFA4003E1B8A
:1017B0003000FEF701FE054B30601B78371D002B13
:1017C00006D0009EFEF765FFE47D00003C0200208D
:1017D0002B68019A1C121340E64A9B009B58043563
:1017E000FEF788FF039A3B1D0493E34C9B1ADB2B07
:1017F00004DD1A23009E2370FEF74BFF02F0B4F8BD
:1018000001234000184323783860002B03D0009E4A
:10181000049FFEF73EFF2B68019A1C121340D54A25
:101820009B009B58049F0435FEF764FF039A3B1D01
:101830000493D14C9B1ADB2B04DD1A23009E2370EA
:10184000FEF727FF02F086F8CC4B4000184001233A
:10185000184323783860002B03D0009E049FFEF7C6
:1018600018FF2B68019A1C121340C24A9B009B5818
:10187000049F0435FEF73EFFA4003E1B3000FEF738
:10188000E5FDBD4B30601B78371D002B02D0009E5C
:10189000FEF7FFFE2B68019A1C121340B54A9B000D
:1018A0009B580435FEF726FFA4003F1B3800FEF7C7
:1018B000E5FDB14B1B78002B02D0009EFEF7E9FE40
:1018C0002B68019A1C121340AA4A9B009B580435AE
:1018D000FEF710FFA300FB1A0493012320001A0057
:1018E0000499FEF71FFEA64C2068643001F080FBCF
:1018F000002816D0029B21685A78A24801F0F7FD13
:1019000015E0A300FB1A0493200001230022049990
:10191000FEF708FE9A4C2068643001F069FB00284D
:1019200002D1043DFEF7C9FE964801F07BFC01237D
:10193000029A137002F00EF8C8222368D200063310
:1019400053431818029B5860FEF7B8FEFEF762FE7C
:10195000894BA4001B783E1B3060371D002B02D042
:10196000009EFEF796FE2B68019A1C121340814AD6
:101970009B009B580435FEF7BDFEA4003E1B3000C3
:1019800002F026F87C4B30601B78371D002B02D00C
:10199000009EFEF77EFE2B68019A1C121340754ACA
:1019A0009B009B580435FEF7A5FEA4003E1B3000AB
:1019B00002F010F8704B30601B78371D002B02D0FE
:1019C000009EFEF766FE2B68019A1C121340694ABE
:1019D0009B009B580435FEF78DFEA4003E1B300093
:1019E00001F0FAFF644B30601B78371D002B02D0EA
:1019F000009EFEF74EFE2B68019A1C1213405D4AB2
:101A00009B009B580435FEF775FEA4003F1B380071
:101A100002F000F8584B1B78002B02D0009EFEF716
:101A200038FE2B68019A1C121340524A9B009B58A7
:101A30000435FEF75FFEA4003E1B300002F00CF8F8
:101A40004D4B30601B78371D002B02D0009EFEF7F7
:101A500020FE2B68019A1C121340464A9B009B589B
:101A60000435FEF747FEA4003F1B380002F026F8BD
:101A7000414B1B78002B02D0009EFEF70AFE2B681C
:101A8000019A1C1213403B4A9B009B580435FEF7F9
:101A900031FE0121200001F0F9FF374B1B78002BAC
:101AA00002D0009EFEF7F5FD2B68019A1C12134030
:101AB000304A9B009B580435FEF71CFE0021200095
:101AC00001F0E4FF2C4B1B78002B02D0009EFEF7A8
:101AD000E0FD2B68019A1C121340264A9B009B587C
:101AE0000435FEF707FEA4003E1B300002F004F8A8
:101AF000214B30601B78371D002B02D0009EFEF773
:101B0000C8FD2B68019A1C1213401A4A9B009B586F
:101B10000435FEF7EFFDA4003E1B300002F000F894
:101B2000154B30601B78371D002B02D0009EFEF74E
:101B3000B0FD2B68019A1C1213400E4A9B009B5863
:101B40000435FEF7D7FDA4003F1B380001F0C2FFAB
:101B5000094B1B78002B02D0009EFEF79AFD2B68E4
:101B6000019A1C121340034A9B009B580435FEF750
:101B7000C1FDC046E47D00003C020020FEFFFF7F67
:101B80004402002048020020A4003F1B380002F05D
:101B9000E7FCD84B1B78002B02D0009EFEF779FDA6
:101BA0002B68019A1C121340D34A9B009B580435A2
:101BB000FEF7A0FDA4003E1B300002F023FDCD4B3C
:101BC00030601B78371D002B02D0009EFEF761FDB0
:101BD0002B68019A1C121340C74A9B009B5804357E
:101BE000FEF788FDA4003F1B380002F065FCC14BE6
:101BF0001B78002B02D0009EFEF74BFD2B68019A4C
:101C00001C121340BC4A9B009B580435FEF772FD22
:101C1000A4003E1B300002F065FCB64B30601B7820
:101C2000371D002B02D0009EFEF733FD2B68019A72
:101C30001C121340B04A9B009B580435FEF75AFD16
:101C4000A4003F1B380002F05BFAAA4B1B78002B64
:101C500002D0009EFEF71DFD2B68019A1C12134056
:101C6000A54A9B009B580435FEF744FDA4003F1B8A
:101C7000380002F05BFA9F4B1B78002B02D0009ECD
:101C8000FEF707FD2B68019A1C1213409A4A9B002D
:101C90009B580435FEF72EFDA4003F1B380002F0D0
:101CA00055FA944B1B78002B02D0009EFEF7F1FCF6
:101CB0002B68019A1C1213408F4A9B009B580435D5
:101CC000FEF718FDA4003F1B380002F067FA894BAD
:101CD0001B78002B02D0009EFEF7DBFC2B68019ADC
:101CE0001C121340844A9B009B580435FEF702FDEA
:101CF000A300FE1A31002000049302F00DFD049BA6
:101D00003060FF1A7B4B04371B78002B02D0009EFB
:101D1000FEF7BFFC2B68019A1C121340764A9B0009
:101D20009B580435FEF7E6FCA300FE1A31002000A4
:101D3000049302F0F9FC049B3060FF1A6D4B0437EA
:101D40001B78002B02D0009EFEF7A3FC2B68019AA3
:101D50001C121340684A9B009B580435FEF7CAFCCE
:101D6000A300FE1A31002000049302F0E5FC049B5E
:101D70003060FF1A5F4B04371B78002B02D0009EA7
:101D8000FEF787FC2B68019A1C1213405A4A9B00ED
:101D90009B580435FEF7AEFCA300FE1A310020006C
:101DA000049302F055FB049B3060FF1A514B04373B
:101DB0001B78002B02D0009EFEF76BFC2B68019A6B
:101DC0001C1213404C4A9B009B580435FEF792FCB2
:101DD000A4003F1B380002F009FA464B1B78002B89
:101DE00002D0009EFEF755FC2B68019A1C1213408E
:101DF000414A9B009B580435FEF77CFCA300FF1A68
:101E00003900200002F0A4FA3A4B1B78002B02D0D4
:101E1000009EFEF73EFC2B68019A1C121340364AC6
:101E20009B009B580435FEF765FCA4003E1B300068
:101E300002F05AFA2F4B30601B78371D002B02D06E
:101E4000009EFEF726FC2B68019A1C1213402A4ABA
:101E50009B009B580435FEF74DFCA300FF1A390088
:101E6000200002F023FA234B1B78002B02D0009EA7
:101E7000FEF70FFC2B68019A1C1213401E4A9B00B0
:101E80009B580435FEF736FCA300FF1A39002000EA
:101E900001F032F8174B1B78002B02D0009EFEF7A2
:101EA000F8FB2B68019A1C121340134A9B009B58A5
:101EB0000435FEF71FFCA300FE1A31002000049336
:101EC00001F01AF8049B3060FF1A0A4B04371B78A4
:101ED000002B02D0009EFEF7DCFB2B68019A1C123F
:101EE0001340054A9B009B580435FEF703FC07B0DE
:101EF000F0BDC0463C020020E47D00000023F7B5A1
:101F00005A1E0192002B07DA01F0A6FF01F060FAD9
:101F100001F012FB6423019300263000194B19686D
:101F20008E4201DB019BEBE7174B1A6801329142AD
:101F300000DC0022F0241A601D68144F6C43E35D3E
:101F4000002B1DD0E419022B16D0012B0ED1002836
:101F500001D101F0FFFCF0226A430C4B0C499B18A5
:101F60005B68C31A8B4201D80223BB54F0235D4344
:101F7000064BEB5C022B03D12000FEF763FBD1E79D
:101F80000136CBE74002002000000020E0110020D5
:101F90009F860100054B01211A68054B1A6000233A
:101FA000044AD1500433642BFBD1704794050020C0
:101FB0008C0500203823002000B59BB002000549A5
:101FC00001A805F05FF801A801F048F901F0B4FAA2
:101FD000FCE7C0462480000037B5174D0400286890
:101FE000002801D004F042FCA400200004F034FCDE
:101FF0002860002801D1114809E001AB984208D2BD
:102000000F4B02196B440193934202D20D48FFF724
:10201000D3FF042802D808302860083C2B680A4AFD
:102020001C191360094B01211C600023084AD15080
:102030000433642BFBD137BD9405002035800000AC
:102040001CFCFFFF658000008C050020900500202F
:102050003823002070B50D4D0D4E2B684C1CA4008C
:1020600036681C19B44203D90A20FEF7CDFA0BE0FA
:102070002C601D00AC4201D904C5FBE70F22090109
:10208000104008431860180070BDC0468C05002041
:10209000900500200322CB1C70B50C00D91711400D
:1020A000C9180500891000220420FFF7D3FF002380
:1020B000A34204DAE95CC21811710133F8E7E14385
:1020C0000023C917214041180B7170BD10B583075B
:1020D00006D1042804D90F2304C81340042B03D0CD
:1020E0000E20FEF791FA014810BDC0466C81000039
:1020F00030B502248025094B094AED009C505C59FB
:10210000002CFCD0A124E400884204D28025ED00FC
:1021100018514019F8E70021995030BD00E0014006
:102120000405000010B5002804D19020922100027F
:10213000890203E0922080218002C902FFF7D8FFC4
:1021400010BD002802D092239B0201E090231B02C5
:102150001B6800201A0E532A01D11B02180A70476F
:1021600030B501248025064A064BED00D450545961
:10217000002CFCD001600021014AD15030BDC04686
:1021800000E001400405000010B5002802D09220B4
:10219000800201E090200002A6230902DB05090A63
:1021A0001943FFF7DDFF10BDF0B5012480250300C2
:1021B0000F4F08000F49ED007C507C59002CFCD0DB
:1021C0009C46002810DD5478167893782402344316
:1021D0001B0423431C00D37801381B0623436446A9
:1021E00008C40432A446ECE700237B50F0BDC0468F
:1021F00000E001400405000070B505004B680A00CE
:102200009C1C2100FFF7D0FFA000281870BD000023
:10221000154B1B68002B04D080219223C9029B021E
:1022200003E09221902389021B02002807D1191D87
:102230005B6802001B0E522B14D10A0012E0002230
:1022400081420FD903681B0E522B0BD14368023316
:102250009B00C318994205D91A68110E0022522911
:1022600000D11A0010007047980700208022F0B5B6
:10227000520085B00021624804F00BFB802200214F
:102280005200604804F005FB5F4B1B681A00029384
:1022900053425A4110000392FFF744FF029B002B68
:1022A00001D15A4C00E05A4C0020FFF7B1FFFF2744
:1022B0000500002D00D194E02B681A121B143A403F
:1022C0003B4001921A000A3A092A43D84C4B019A22
:1022D000995C002900D07FE010224E4804F0D9FA22
:1022E0002E00336801991A123A40914217D11A14FC
:1022F0003A400B2A06D0132A0CD00A2A0FD1454B9C
:102300001E600CE03B40022B09DC424A9B00D318C4
:102310005E6004E0102200213E4804F0BAFA30006A
:10232000FFF776FF061EDCD13A4B196800290FD063
:102330002000FFF761FF0400374E3168002903D009
:102340002000FFF759FF0400344B0436B342F4D1A8
:102350002B4B3EE0143B092B3ED82A4B019A995C4B
:10236000002939D108222E4804F093FA2E00336850
:102370001A143A40152A0BD01D2A11D0142A14D150
:10238000019A1B123B409A420FD1254B1E600CE074
:10239000019A1B123B409A4207D1214B5E6004E038
:1023A000082200211E4804F074FA3000FFF730FFC5
:1023B000061EDCD11A4E3168002909D02000FFF733
:1023C0001BFF71680400002902D0FFF715FF04000D
:1023D0000C4B0121019A99542800FFF719FF0500C1
:1023E00067E70298FFF7ADFE411C0398FFF7CCFEAC
:1023F000054B039A1A600B4B1C6005B0F0BDC0463C
:102400009806002098050020980700200448020044
:10241000049000009C230020A0230020AC23002077
:10242000AC2300209C07002070B50020FFF789FE38
:1024300004000120FFF785FE844200DA04000A4B05
:102440001E687542754128001D60FFF76BFE002E67
:1024500001D0064B00E0064B064A2800611C1360C1
:10246000FFF792FE70BDC046980700200490000060
:10247000044802009C070020F8B50020FFF761FE29
:1024800007000120FFF75DFE3E00224D0643224C6F
:102490000CD180219020C9020002FFF729FE012102
:1024A0003000FFF771FE2E601C4B2FE0874208DDE5
:1024B000002392212B60194B89022360236800209E
:1024C00011E0012380212B60154BC9022360F5E741
:1024D0001A68551C18D0120E522A07D101205A68CA
:1024E000023292009B188B42F2D311E0002800D0F8
:1024F00023600C4C0C49200004F0F0FD200001F09A
:102500003BFAFFF791FF04E0002802D0236000E0CF
:102510002160F8BD980700209C070020049000006F
:1025200004480200F0230020DD800000F0B585B0F3
:10253000039203220333DC1714402A4EE3189C1045
:10254000336801900291002B02D08022D20201E078
:1025500092229202244FA51C3B68AD005B199A425F
:1025600017D2FFF783FE3368002B02D08022D202FD
:1025700001E0922292023B685B199A4209D21B4CFD
:102580001B49200004F0AAFD200001F0F5F900200D
:1025900026E0029B3E681B06190C6B461A7BA4239F
:1025A000DB051343019A0B431104FF22120411406F
:1025B00019433000FFF7D4FD3300301D08332100EC
:1025C00001933B60FFF7CCFD002C04D00A9A210058
:1025D0000198FFF7E9FD3000019B083D5D193D6062
:1025E00005B0F0BD980700209C070020F0230020D4
:1025F0000681000070B59AB0FFF73EFFFF221F4C26
:10260000D2000021200004F044F90020FFF700FE72
:10261000FF25002600281AD003681A142A400A2A27
:1026200008D11A122A40FF2A0ED0D200A1180B712D
:10263000A05009E0132A07D11B122B40FF2B03D017
:10264000DB00E2181671E650FFF7E2FDE2E7FF213A
:102650000200C900235808305D1EAB41D2188842E1
:10266000F8D1074901A804F00DFD01A800F0F6FD1E
:10267000044800F0F3FD1AB070BDC046401B0020B6
:102680002D8100004581000000220121094B5A6084
:10269000094A51605A68002AFCD00022C021054B2B
:1026A00049001A61044B01329A60044B01325A50BE
:1026B0001A607047FC1000400010004000E100E08C
:1026C0000222064B0121DA670022054B5A61054AB6
:1026D00011615A69002AFCD07047C04604E100E04D
:1026E000FC1000400010004010B5054B1A781C008B
:1026F000002A01D0FFF7E4FF0023237010BDC0467D
:1027000028080020024B1868012340001843704736
:102710002408002000487047D8230020024B186886
:1027200001234000184370477400002070B5040076
:102730000D00160001F018F98023012200215B052D
:102740005B6E6270E270020AA271020CE2711A0AF8
:1027500060716372000EA2721A0C1B0E2670257136
:102760002072A170E272237370BD0000124B10B58D
:102770001B68124C5A1C0FD0114C002B0CD0114C62
:10278000012B09D0104C022B06D00D4C042B03D08A
:102790000E4C052B00D10B4C21000D4804F09EFC83
:1027A000200004F0A3FC0300042204339B08094822
:1027B0001B011343036010BD780000200F8200004E
:1027C000088200001A8200001F82000014820000AC
:1027D000B8230020B423002070B5214C2278002AB1
:1027E0003DD1204B01215A608022D20511605A68E8
:1027F000002AFCD0002207201B4B1C4901255A50FF
:102800000439585008315A5019481A4958501A4931
:102810001A485A501A495A50A622D2009D500822EE
:1028200018495A5004315850022017495850174837
:10283000174958501748043958501820164958500D
:10284000C12189005A500539FF395A5808380243C6
:102850005A50124A12499950FFF716FF257070BD61
:1028600028080020FC000040001000400C0500007B
:10287000746962751C050000240500002000040234
:102880002C0500001405000034050000FFFF0000C7
:102890003C05000021100100540500000405000063
:1028A000A007002010B500280EDD0C68E3070BD54B
:1028B0006410FF2C08D8054B1B78002B01D1FFF7C3
:1028C0008BFF034B034AD45010BDC046280800209C
:1028D000240500000010004013B5002815DD0C6829
:1028E000E30712D5082209496846641003F0C8FFBF
:1028F000072C0AD8064B1B78002B01D1FFF76CFF81
:102900006B46044A1957044BD15016BD0082000093
:1029100028080020001000400C05000010B5002819
:1029200013DD0C68E30710D56410532C0DD8074B4A
:102930001B78002B01D1FFF74FFFFFF7C1FEA1234A
:10294000034ADB00D450FFF79FFE10BD280800208B
:102950000010004070B50E4B06001B78002B01D113
:10296000FFF73AFF00200B4D2C7884420ED00A4B23
:10297000202219780323091B1940084B49015918D3
:10298000300003F07DFF0120013C2C7070BDC0467B
:10299000280800202908002020080020A007002087
:1029A000002330B589B0984226DD03240D682C4001
:1029B0009C4221D12300042D1ED90F212A681140E9
:1029C000062919D112091F2A16D96846FFF7C2FF36
:1029D0002300002810D06B46012019780123A14262
:1029E00003DB6B461B5D5B000343A200AA180134A6
:1029F0005360202CF2D10423180009B030BD000030
:102A0000F0B5424B8BB01B78002B01D1FFF7E4FEF1
:102A100002AD2800FFF79EFF002870D02B780B2B0B
:102A20006DDD6B78012B6AD1EA780023012A66D12B
:102A3000374F384C3B6023712B79374A1360002B9A
:102A40000ED115256D446A782878AB7812020243BE
:102A50001B0413431A00EB781B0613433B6050E042
:102A6000012B10D115266E4472783078B37812029B
:102A700002431B0413431A00F3781A261B06134360
:102A80003B606A7C25E0022B02D16A7B162620E09F
:102A9000042B0DD1152108226944684603F0F0FE8D
:102AA0000098019902F0A4F803F016FE386028E0BF
:102AB000052B26D1152108226944684603F0E0FE63
:102AC0000098019902F094F803F006FE1E26386083
:102AD0006A7D6E44132A00DD13220023934204D042
:102AE000F05CE11808710133F8E704200021E218D6
:102AF00004339B101B0103431171236003E000208A
:102B000001E00022E9E70BB0F0BDC0462808002034
:102B100024080020D82300207800002010B5041ECF
:102B200026D0144B1B78002B01D1FFF755FEFFF781
:102B3000C7FD00201049114A114B8C5058600130DC
:102B4000086059680029FCD000200D4908610A4935
:102B50000130886019690029FCD00A4B0A491B78AA
:102B60005B01CB1804498B50FFF7AAFDFFF78CFDE2
:102B700010BDC046280800200010004004050000D9
:102B8000FC10004020080020A007002030B589B0CC
:102B900000281EDD03230A6813401AD1042A18D91D
:102BA0000F2011680840062813D109091F2910D9E0
:102BB00001240133990051580020214201D04910CD
:102BC000C8B26D46591E6854202BF2D16846FFF7F3
:102BD000A5FF09B030BD30B589B0002826DD0868F2
:102BE000830723D1042821D90F2302681340042B23
:102BF0001CD1FFF76BFA050004F078FA041E122CC2
:102C000000DD1224220002210D326846FFF78EFDFE
:102C10006B465C730023A34205DA1A00E95C6A4440
:102C200091730133F7E76846FFF778FF09B030BDCD
:102C300070B50C0088B0012833DD0868830730D1F7
:102C400004282ED90F2302681340042B29D14B6886
:102C5000DB0726D5FFF73AFA060004F047FA646866
:102C6000050064100E2800DD0E252A000121113216
:102C70006846FFF75BFD6B466A465C7323129373ED
:102C80002314D3730023240E14745574AB4205DA55
:102C90001A00F15C6A4491740133F7E76846FFF764
:102CA0003DFF08B070BD30B589B0002814DD0C6858
:102CB000E30711D5102200216846FFF737FD6B4668
:102CC0006A4665105D73684663122D0E6414937333
:102CD000D4731574FFF722FF09B030BD184B10B53F
:102CE0005A681849002A03D000225A6001328A60CB
:102CF0001B691448002B22D00023114A1361802243
:102D0000D2008458104A012C16D1A923DB00C358E5
:102D10005B4213600D4A1378032B01D80133137003
:102D200003220B480378013313400A4A03705B0106
:102D3000D318094A8B5000E0136001238B6010BD4B
:102D4000FC10004000100040740000202908002002
:102D500020080020A00700200405000010B5034A49
:102D60000E21034800F0B4F810BDC0460400002056
:102D700026820000044A05491368C85401339B05A4
:102D80009B0D13607047C046300C00202A080020BD
:102D9000114A70B51368114C984211DA015D451C57
:102DA000FA39012906D8AB4206DD211849780139E4
:102DB0001F2901D92800EFE70100251A461C02D17E
:102DC0000023136006E0665C6E5401318B42FADC2E
:102DD000181A106070BDC046340C00203C0C002056
:102DE00010B500F0B7FD064B1A68904201D20022E0
:102DF0001A601B68C01A034B83428041404210BDD9
:102E0000380C0020204E000010B5094C094A2368F8
:102E1000126893420BD0084AD05C00F0D7FE00281D
:102E200005D0236801339B059B0D2360EDE710BDA2
:102E30003C100020300C00202A08002010B50400AF
:102E4000064B074A1B6812689B1ADB439B059B0DC8
:102E5000A34202DAFFF7D8FFF2E710BD300C0020E2
:102E60003C100020F7B506000191151E2FD05768C1
:102E7000B800441C0630FFF7E1FFFB20FFF77AFFA4
:102E80001C20FFF777FFF0B2FFF774FFE0B22412C7
:102E9000FFF770FFE0B2FFF76DFF6B461879FFF7A1
:102EA00069FF0026BE4212DAB300EB189C680136B7
:102EB000E0B2FFF75FFF2012C0B2FFF75BFF201404
:102EC000C0B2FFF757FF200EFFF754FFEAE7F7BD48
:102ED00070B5074D2C68092C08DC0C236343054EA4
:102EE00001349851F31859609A602C6070BDC04647
:102EF0004010002054240020F0B589B004900E004A
:102F000001284BDD284B08680293830709D1042868
:102F100007D90F2302681340042B02D1FFF7D6F81C
:102F20000290214B70680393830709D1042807D9C5
:102F30000F2302681340042B02D1FFF7C7F8039058
:102F400000271A4B1A4D1B680593059B9F4225DAF3
:102F50002B1F0299186804F0B7F800281BD12B68C2
:102F60006C6806930190019B069A934213DA2068DD
:102F70000399079404F0A8F80834002807D1310019
:102F80000498079B08315B680238984709E0019B69
:102F900001330193E7E701370C35D6E71B20FDF736
:102FA00033FB09B0F0BDC0466C810000401000202A
:102FB0005824002010B501F03FFA00F0C7FD00F0E2
:102FC00033FEFFF7CBFE01F09BFA01F0D1FB10BD01
:102FD000962210B512010021034803F05AFC00228A
:102FE000024B1A6010BDC046E011002040020020D4
:102FF000064B074A1B6812689B1ADB439B059B0D17
:103000000122834200DC002210007047300C0020B7
:103010003C100020F8B505000C0016001F1E0ED154
:103020000320FFF7E5FF002827D0FA20FFF7A2FED4
:10303000E8B2FFF79FFEE0B2FFF79CFE1DE0501DD7
:10304000FFF7D6FF002818D0FB20FFF793FEE8B269
:10305000FFF790FEE0B2FFF78DFEF0B2FFF78AFEB9
:103060003012C0B2FFF786FE3C00E31B9E4204DD37
:103070002078FFF77FFE0134F7E7F8BD70B5002434
:10308000F0250B4B1B689C420EDA2A006243094B69
:10309000D3181A78002A05D05978002311201A0075
:1030A000FFF7B8FF0134ECE7FFF792FF70BDC046B1
:1030B00040020020E01100200123F3B50400FFB01E
:1030C0000D0010001A420DD002AA1370431002A97D
:1030D000537042121B0E40148A700B71C8700B00A3
:1030E000052273E0032313401ED1042A1CD90F22AA
:1030F00001680A40042A17D1023302AA1370FEF7AE
:10310000E5FF060003F0F2FFF823FF33984200DDED
:1031100018000023834205DA01335A1EB25C02A96B
:10312000CA54F7E7421C50E0042801D0002809D116
:10313000032302AA0438137043424341537013001F
:10314000022243E0002B45D1042843D90F21026815
:103150001140052912D1043302A90B70F82312097A
:10316000FF3392009A4200DD1A00002393422BDACB
:103170000133C118C97802AEF154F7E7062929D105
:1031800001390E00120956430196F826019FFF36B9
:10319000B7421FDC02AE31700136934213DA0127C9
:1031A000013399004158394201D0394100E00A49C0
:1031B000012737700F127170B7700F14090EF77076
:1031C00031710536E9E7019A013202AB290020008E
:1031D000FFF720FF7FB0F3BD19FCFFFF70B5F023B0
:1031E000050000240D4A1800604380184178A94268
:1031F00003D001340A2CF6D10FE0F022002103F0B5
:1032000048FB074A1368013BA34200D11460002326
:1032100029001A001120FFF7FDFE70BDE01100200B
:103220004002002010B5B2B002236A4604001370B9
:1032300003F05CFFC72800DDC7200023834205DAC6
:10324000694601335A1EA25CCA54F7E7421C6B461A
:10325000FE211420FFF7DEFE32B010BD10B5B2B073
:1032600002236A460400137003F040FFC72800DD04
:10327000C7200023834205DA694601335A1EA25C47
:10328000CA54F7E7421C6B46FF211420FFF7C2FE29
:1032900032B010BDF7B5234B06001B68F020009339
:1032A00000232149009A93420ADA02005A438A18FD
:1032B0005478B44202D11278002A31D10133F1E7B7
:1032C0000024F0231A00624301920199164A55180E
:1032D0002F78002F06D001340A2CF3D11348FFF7C2
:1032E000BDFF1DE0F0223900280003F0D2FA0223CE
:1032F0000D4A0199EB6053540D4AF1008A58009B26
:103300006E70AE70AA602F616F61A34202DC054B44
:1033100001341C60002331001A001020FFF77AFEF0
:10332000F7BDC04640020020E0110020E18200000D
:10333000401B002010B5FFF7A1FE0024064BE20061
:10334000D3181B79043B012B02D8E0B2FFF7A2FF90
:103350000134FF2CF2D110BD401B0020F7B50E0048
:1033600000247F250190194BE200D1180979062924
:1033700001D0032926D1985883682B401C2B21D1DA
:10338000C3681A002A40042A1CD102692A40192A5B
:1033900018D11B0A01339B000C30C018FEF796FEB3
:1033A000070003F0A3FE0023B0420BD19E4206DDCE
:1033B000019AF95CD25C914204D10133F6E7E0B2A4
:1033C000FFF768FF0134FF2CCDD1F7BD401B002073
:1033D00070B500F0BFFA184B1A68904201D2002273
:1033E0001A601A681549821A8A4223D91860002087
:1033F00000F082FB44424441604207240443002021
:1034000000F08EFB002810D0082600250C4BEA00A7
:10341000D3181B799C4201D0B34202D1E8B2FFF726
:1034200039FF0135FF2DF1D104E0631C02D00126E4
:103430007642EAE770BDC0462C0C00200F27000042
:10344000401B002037B500240500FFF717FE01A838
:10345000019400F03FFB200000F068FE00F0FCFC4F
:1034600000F072FB00F071FB00F038FF00F09EFAF4
:103470000548FFF7F3FEA54204D0FEF78BFD034895
:10348000FFF7ECFE37BDC046F68200000E83000059
:10349000002310B501001A001120FFF7BBFD10BD7D
:1034A00007B56B46197069465A7013128B70131466
:1034B000120ECB700A716B46010005221320FFF734
:1034C000A9FD07BD10B50A0001001220FFF7F4FDA9
:1034D00010BD70B5050008000C003230FFF7AEFCDF
:1034E0002B00220000211B20FFF794FD70BD10B5BA
:1034F0000C000300110014202200FFF78BFD10BD0B
:1035000070B506000020FEF783FE0024FF2500288A
:1035100010D003681A142A40152A05D11B122B401B
:10352000B34204D1040002E01D2A00D10024FEF7BA
:103530006FFEECE7200070BDF0B580279DB0FFF76F
:1035400063FCB94DB94C2868FF00391A201800F007
:1035500023FB2B680600C3182B60002B00D1DBE196
:10356000002E0DDD2868391A201800F015FB2B6895
:1035700006001B182B6000F0EDF9AD4B1860EFE76B
:103580002378FA2B00D00CE12B68022B06DCFFF726
:1035900027FC002800D1BFE10120B8E16078A578C0
:1035A0000238182800D9FAE002F06AF80D1E222627
:1035B0002932F93D676F7589DAEFF9F9F9F9F9F907
:1035C000F9F9F9F9F300FF2D00D1E8E02800FFF741
:1035D00005FE00229749EB005A50CB181A712900BA
:1035E0000092130013204DE02800FFF753FED6E0B1
:1035F0002800FFF7F3FDD2E0FFF79CFECFE0FFF7D6
:103600003DFD0020FFF71EFF8B48FFF727FEC6E0B9
:10361000182D00D9C3E0894BAA00D25829001520E3
:10362000FFF74AFDBBE000242000FFF769FF071EFB
:1036300003D10134192CF7D1B1E0083003F056FD65
:1036400006000530FFF7FAFBFB20FFF793FB1D2078
:10365000FFF790FBE0B2FFF78DFBF0B2FFF78AFBBC
:103660003012C0B2FFF786FB0025AE42E1DD7B19C8
:10367000187AFFF77FFB0135F7E700211D200B00CB
:103680000A000091FEF752FF89E000222900009213
:1036900013002720F6E700F077F903AC684A6421AD
:1036A0000090684B200003F0BBFC02232000237035
:1036B00003F01CFD23000200002116206DE0002411
:1036C0005C4AE300D558002D46D06B689E00701D03
:1036D000FFF7B4FB2B000025320008332100012046
:1036E000FFF798FC0020FEF793FD2E002F00002826
:1036F0001DD0FF2103681A120A40A24214D11A14E5
:103700000A400B2A07D10B400DD0012B09D0022B08
:1037100000D1FFE008E0132A06D100252E002F007B
:1037200002E0060000E00700FEF772FDDFE7002E72
:1037300004D0320001212000FFF794FB002D04D0BB
:103740002A0002212000FFF78DFB002F04D03A0051
:1037500000212000FFF786FB0134FF2CB0D11EE0D2
:10376000FFF78CFC00250024290000942300220090
:1037700013200135FEF7DAFEFF2DF4D1FF222100E0
:10378000D2002C4803F085F809E00120FFF75AFE2B
:1037900005E0002329001A001A20FFF73BFC032054
:1037A000B5E0FB2B00D0F7E62A68042A00DCEEE641
:1037B0002679E078244B360206439E4200DDEBE694
:1037C000331D9A4200DCE2E6E35CFE2B00D0E3E628
:1037D0006078A578731E1C2868D007D8082835D0D3
:1037E0001B285ED0012800D090E007E01E2800D101
:1037F0007EE066D31F2800D180E087E0FF2D00D156
:1038000084E02800FFF7EAFC67790634B31E29003C
:1038100000943A000A20FEF789FE064BED00E850BE
:103820005D192F7172E0C046340C00203C0C002062
:10383000380C0020401B00201E830000382300208D
:103840003583000030830000F6030000182D5DD89A
:103850006079022813D003281BD0012856D1A71D58
:103860007A78A479BB78120222431B0413431A000E
:10387000FB78AD001B0613435B0003430EE0002BF7
:1038800044DDB11EA01DFEF705FC244BAD00E85041
:103890003CE0A379AD005A1E93419B001F4AAB50F8
:1038A00034E0601D1900FFF759FD2FE0FF2D2DD0EA
:1038B0006279022A2AD80634B31E009429000B200C
:1038C00022E0632B00DD6323002203A8934204DD82
:1038D000A118497981540132F7E7D9430022C91769
:1038E000194041180A7001330090290015200BE09F
:1038F00005340094002229001E2005E0042B05D188
:103900000022290005340094FEF710FE701DFFF719
:103910003FFA01E0050007E71DB0F0BD38230020A5
:10392000002070470020704700207047002070473B
:1039300001220020054B06491A615850033004311A
:1039400058508018083158501A6070470080004065
:10395000040500000122034B1A64A822D2009858E3
:103960007047C0460080004010B5FFF7F3FFFA2112
:10397000890001F08FFE10BD10B50100014801F073
:1039800033FC10BD6C1100200048704744830000D8
:1039900070B5054E0400335C0D008B4202D001F07F
:1039A0004BFB355570BDC0464410002070B5002457
:1039B000064D635D012B05D10021200001F03CFB89
:1039C0000023635501341D2CF2D170BD441000203A
:1039D0000D2070473B207047036870B55B100120D5
:1039E000052B12D8094A9B009C58094D2B5D002BD2
:1039F00005D00021200001F01FFB00232B552000E3
:103A000001F0C4F901234000184370BD7483000025
:103A10004410002070B5036845685C106D1004D434
:103A20000B4B9D4202DD1D0000E000251C2C0DD833
:103A3000084E335D012B05D00121200001F0FCFA76
:103A4000012333552900200001F02EFA70BDC04635
:103A5000FF0300004410002070B5046864101C2CA3
:103A60000FD8094D2B5D002B05D00021200001F05F
:103A7000E3FA00232B55200001F012FB0423012858
:103A800000D00023180070BD4410002070B5040061
:103A90000D001C280ED8084E335C012B04D00121E8
:103AA00001F0CAFA01233355290020004D1EA94117
:103AB00001F0E0FA70BDC04644100020436810B524
:103AC000191F4A424A41006811004010FFF7DEFF0B
:103AD00010BD000037B569460200064B684630CB82
:103AE00030C11368042B02D100F030FB01E000F07C
:103AF00055FB37BD3C83000010B5084C6379002BA3
:103B000005D00021052001F097FA002363710520FC
:103B100001F0C6FA43425841800010BD4410002015
:103B200010B5084CE37A002B05D000210B2001F0E2
:103B300083FA0023E3720B2001F0B2FA43425841AA
:103B4000800010BD441000207047704710B5034A34
:103B500004210348FFF7BCF910BDC0467C000020DB
:103B600036820000E12110B54902094801F083FBCB
:103B7000FFF7DEFE0A2001F003F90023FF21054ACA
:103B8000995401331D2BFBD100F0A8FB10BDC0469A
:103B90006C11002044100020F8B50B4E07003000D7
:103BA0000D0001F0A7FB041EAC4200DD2C003D001F
:103BB000EB1B9C4205DD300001F0A6FB28700135AF
:103BC000F6E72000F8BDC0466C11002010B50100DA
:103BD000014801F057FB10BD6C1100200020704718
:103BE00010B51E20FCF710FD10BD10B51E20FCF70F
:103BF0000BFD10BD10B51E20FCF706FD002010BD0A
:103C000010B51E20FCF700FD10BD10B51E20FCF7FE
:103C1000FBFC10BD10B51E20FCF7F6FC10BD10B566
:103C20001E20FCF7F1FC10BD10B5034A0821034823
:103C3000FFF74EF910BDC0469C0000208C830000A9
:103C40000123034A1360034A1068984018437047E1
:103C50006C10002074100020202800D90020084B90
:103C60008000C25801239340064A07491360074A5F
:103C70001160074A07491160074A13607047C04640
:103C800054880000681000200805005084100020AF
:103C90007C1000200C05005018050050F0B5EFF323
:103CA00010810123194083F31088134E134AB44640
:103CB0001268013A9340124A1468124A1568124A6F
:103CC000002B15D0166803420BD02660C046C046B4
:103CD000C046C046C046C046C046C04616682E60B4
:103CE00004E067463E601668084F3E605B08E7E701
:103CF00081F31088F0BDC04608050050E4000020A4
:103D0000841000207C100020681000200C0500505A
:103D100030B585B001AD0C220649280002F0B0FD97
:103D20000024285D01210134FFF732FE0C2CF8D16C
:103D300005B030BD02840000F0B53B4C85B02100D9
:103D400003220C31684602F09BFD210009220F314D
:103D500001A802F095FDFFF707FE344B344CC01864
:103D60002368984201D2002323602568002D3ED1AC
:103D70002E006B4604339F5D01213800FFF708FEDB
:103D800001360121380001F075F9092EF1D1002624
:103D90006B469F5D01213800FFF7FAFD01360021D7
:103DA000380001F067F9032EF2D1C82080000138F5
:103DB000C046C046C046C046C046C046C046C046D3
:103DC000C046C046C046C046F1D100210420FFF7DE
:103DD000DFFD00266B460021985D0136FFF7D8FD18
:103DE000032EF7D1FFF7C0FD1330206019E0FFF775
:103DF000BBFD23680025984213D3042000F0C6FFC2
:103E00000C4B0D4EC01801D4306000E035603068B6
:103E1000032101F0C9FC00230125084A306023601A
:103E20001360280005B0F0BD0284000010270000D8
:103E300064100020C8FEFFFF741000206C100020EA
:103E400010B50124044001D0441002E00D20FCF71D
:103E5000DBFB200010BD00007FB5A44E3368002BB3
:103E60000BD1A34A1268002A07D1A24B1B68002B72
:103E700000D139E1FFF760FF36E19F4D2A68002A43
:103E80002AD19C4A1268002A07D0FFF755FF002864
:103E900000D129E1FFF73CFF05E0954A1268002AAE
:103EA00001D1002BF6D1924B19681A00002911D0CC
:103EB0003468002C0ED101AD0C22904928001C6002
:103EC00002F0DEFC285D00210134FFF761FD0C2CBF
:103ED000F8D109E13368136000211A2001F0CAF813
:103EE00000211B2001F0C6F800211C2001F0C2F8BF
:103EF0002E68012E56D0022E00D19CE0002E00D05C
:103F0000ECE0013631007A4C03202368994301F03C
:103F1000B1F80420216801400B005942594101F0D9
:103F2000A9F8102123680A200B405942594101F099
:103F3000A1F88021236809010B405942594106200C
:103F400001F098F88021236809020B405942594139
:103F5000072001F08FF88021236849020B40594265
:103F60005941092001F086F88021236889020B401D
:103F700059425941192001F07DF880212368C90276
:103F80000B4059425941182001F074F880232168F0
:103F90001B030B4059425941172001F06BF83100C7
:103FA0001A2099E00221524C172023680B405942F5
:103FB000594101F05FF80821236818200B4059424D
:103FC000594101F057F880212368C9000B4059423C
:103FD0005941042001F04EF88021236849010B402B
:103FE000594259410A2001F045F880212368C9014E
:103FF0000B4059425941032001F03CF880212368CD
:1040000089030B4059425941092001F033F88023BC
:1040100021681B040B4059425941192001F02AF82C
:104020003100062001F026F83100072001F022F8C7
:1040300031001B2050E020212D4C172023680B401D
:104040005942594101F016F84021236818200B40CD
:104050005942594101F00EF88021236819200B4084
:104060005942594101F006F88021236849000B406C
:1040700059425941092000F0FDFF80212368890041
:104080000B4059425941072000F0F4FF802123687A
:1040900089010B4059425941062000F0EBFF802175
:1040A000236849030B40594259410A2000F0E2FFBE
:1040B00080212368C9030B4059425941032000F075
:1040C000D9FF802321685B040B40594259410420E9
:1040D00000F0D0FF01211C2000F0CCFF2B68032151
:1040E000581C01F047FC29607FBDC04678100020B5
:1040F000701000206C10002080100020028400004E
:10410000006810B5C30703D5FFF79AFE054B18608A
:10411000054B1B68002B03D0024B186800F026FBF0
:1041200010BDC046781000208C1000200022054BE6
:1041300010B51A60044B1B68934201D000F014FBC9
:1041400010BDC046781000208C10002070B505000E
:104150000068FFF775FE04006868FFF771FE631ED4
:104160000100042B14D8451E042D11D805226A43E2
:10417000D318012215009D402B00064805682B43EB
:104180000360054B1B68002B02D0200000F0EDFA05
:1041900070BDC046781000208C10002070B505005E
:1041A0000068FFF74DFE04006868FFF749FE631ED4
:1041B0000100042B14D8451E042D11D805226A4392
:1041C000D31801229A401300064802689A43064B0E
:1041D00002601B68002B03D00022200000F0C5FA0B
:1041E00070BDC046781000208C1000202C4BF7B515
:1041F0001B680400002B03D101204042FFF72CFD77
:1042000001262468344219D0FF22631018021204D8
:104210001040FF22611212020A40DBB21043184321
:10422000204B1B68202B06D1B4401F4BA40EA400CA
:10423000E35800021843FFF731FD30E00325254025
:104240002DD1042C2BD90F2322681340062B26D105
:10425000FF27130901933F04019B9D421FDAAB0026
:10426000E3185A68324218D0531018023840FF2120
:1042700084460902501208406146DBB208431843E5
:10428000084B1B68202B06D15200920E064B920061
:10429000D35800021843FFF701FD0135DCE7F7BDF5
:1042A00068100020E4000020308400000B6810B586
:1042B0000200D80701D5581001E001204042182320
:1042C000012A03DD4A68042A00D10833024A136038
:1042D000FFF7C2FC10BDC046E4000020012010B56D
:1042E0004042FFF7B9FC10BD0068F8B5C30702D51E
:1042F000FFF7A6FD0BE0830726D1042824D90F225F
:1043000003681A40042A1FD11B091DD0007903003D
:10431000203B5E2B18D80522002053430B4E9D18DE
:10432000043AAB420CD0052110249F5D3C4200D0E2
:1043300080180139520064100029F7D10133F0E7E9
:1043400001234000184300E00120F8BD3085000043
:10435000F0B5050085B008680C00FFF771FD03900B
:10436000022D08DD6068FFF76BFD0700A068FFF70E
:1043700067FD040001E00124270005236343053B9A
:104380000293012326000193231D9E4234DC3D004D
:104390003B1D9D422BDC731E042B23D86B1E042B6C
:1043A00020D8029B039A591E019B49191A40204BA1
:1043B0000AD001228A4019680A431A601D4B012263
:1043C0001B68002B0ED009E001208840010018680E
:1043D00088431860174B1B68002B03D0310028005E
:1043E00000F0C3F9019B01355B000193D0E7029B0C
:1043F000013605330293C7E73D1D042D15D8012C66
:1044000013D126003300AB40094A11689943094B88
:1044100011601B68002B04D0781D0022210000F0E1
:10442000A4F901340535062CECD105B0F0BDC04629
:10443000781000208C10002010B5034A0121034899
:10444000FEF746FD10BDC046DC0000201A840000C7
:104450000122094B1A60094A1368002BFCD0032281
:10446000074B1B68D8171040C0180123801006386E
:10447000400018437047C04600C0004000C10040E3
:1044800008C500400120704710B501210D20FFF73D
:104490007FFA01210E20FFF77BFA00210F20FFF7A2
:1044A00077FA044C200000F0D5F91021200000F02C
:1044B000EDF910BD9C10002010B504680D20E30735
:1044C00003D56410FF2C03D91720FCF79DF806E0F4
:1044D000FFF7DAFFE1B2024800F0FAF9002010BD60
:1044E0009C10002010B5FFF7CFFF0021034800F01B
:1044F000EFF901234000184310BDC0469C10002076
:1045000010B5034A05210348FEF7E2FC10BDC04682
:10451000EC0000200B870000F7B50F4F06003B684A
:104520000D0001920D4C002B04D1200000F056FA32
:1045300001233B60F1B2200000F0DEFAE9B2200076
:1045400000F00DFA6B462000197900F008FA2000FF
:1045500000F03CFBF7BDC04688100020B0100020E2
:1045600010B501240368234205D04168214202D0DE
:104570008268224201D10D2004E0581049108028A1
:1045800003D91520FCF740F80BE0FF2901D91620CC
:10459000F8E75210FF2A01D91720F3E7FFF7BCFF15
:1045A000002010BDF8B5154F05003B680E00144CF7
:1045B000002B04D1200000F011FA01233B60EDB282
:1045C0002900200000F098FAF1B2200000F0C7F9AD
:1045D0000021200000F09CFA002801D040420CE0AD
:1045E00001222900200000F082FA200000F0ADF93D
:1045F0000028FAD0200000F0ADF9F8BD88100020A6
:10460000B010002010B501240368234202D0416895
:10461000214201D10D2004E058104910802803D90F
:104620001520FBF7F1FF07E0FF2901D91620F8E775
:10463000FFF7B8FF4000204310BD0000002370B515
:10464000344D0400EB5601332BD10D211D20FFF713
:10465000A9FF5A2804D101222A212A703D380AE0F4
:104660000F211920FFF79EFF332807D102235F2275
:1046700020212B701A38FFF74FFF12E00D211E206A
:10468000FFF790FFC7280AD1032300222A21A93867
:104690002B70FFF741FF1B222A211E20EBE700238E
:1046A0002B700023EB56022B06D0032B13D0012BCB
:1046B00026D121001D2010E0012C04D12921192030
:1046C000FFF770FF0DE0032C15D12B211920FFF708
:1046D00069FF043C05E021001E200124FFF762FF72
:1046E00064427F2801DD0138FF3803007F330ADA96
:1046F0007F20404207E0052C02D12D211920ECE754
:1047000001240020644264237F21584301F04CF8C7
:10471000604370BDE800002010B50120FFF78EFF58
:1047200001234000184310BD10B50320FFF786FF9A
:1047300001234000184310BD10B50520FFF77EFF90
:1047400001234000184310BD00207047002070472F
:1047500000207047002070470020704700207047FD
:104760000020704700207047704770477047000076
:1047700010B5034A08210348FEF7AAFB10BDC04646
:10478000140100203B87000010B5FFF7EBF9AF20C4
:10479000C000FDF721FCFEF70DFC0448FEF75EFDAE
:1047A000FDF728FFFEF7C6FD10BDC046F6820000EB
:1047B00010B5FDF7A3FB10BD70B5002504AC24783F
:1047C0000573A94205D10A4B0A4A23210A4801F080
:1047D000D7FF01600949920052589B0002715B5853
:1047E0008371A3005B58856043710223C37170BD60
:1047F000BE87000081870000CC870000548800003D
:10480000037B002B04D14373837303610133037370
:10481000704700001FB50191A02100240068C90065
:10482000D2B24450012A07D0A24203D0032A05D1B4
:10483000042202E0022200E006221343034A8350CE
:10484000034B019AC250012343501FBD5405000081
:104850002405000010B50400FFF7D2FFA122236851
:10486000A179D20099506179064A200099502179A6
:1048700004329950044B19685A689B68FFF7CAFFC5
:1048800010BDC0460C050000901000204BB2002B5C
:104890000CDB80233F290CD81F290CD80F290CD8FA
:1048A00007290CD803290CD81B060BE080239B0496
:1048B00008E0DB0406E01B0504E05B0502E09B0565
:1048C00000E0DB050168014A8B50704724050000B9
:1048D0000368074A99501A00FC32D1680029FCD0BD
:1048E000A321C90058580023C0B2D3607047C04606
:1048F0001C05000007B58022074BD2051A60002274
:104900009A6002321A710F230C3200930349023B62
:104910000348FFF751FF07BD901000200030004012
:104920009C100020F8B505000E0017000024BC42C2
:1049300008D02B68315D1B6828009847002801D0FB
:104940000134F4E72000F8BD704710B51C3000F0CA
:1049500077FC10BD10B51C3000F064FC10BD70B5C4
:10496000437E0D00002B05D06430040000F077FC7E
:10497000002801D0002004E02000290000F043FCC2
:10498000012070BD10B51C3000F060FC10BD0000AF
:10499000F7B50193FA23002504009B0083600D4BBB
:1049A0004560083303601C300F00160000F020FC47
:1049B0002000643000F01CFC074AB600B3582761A1
:1049C0006375019B20009B009B586576A576A375B7
:1049D000FEBDC04634880000548800000123A02298
:1049E000C375837D0C49C133FF33D2059B009950B9
:1049F000437DC133FF339B009950CC210369074AA3
:104A0000490499500521243A9950817D08329950E2
:104A1000417D034A995070470C06000024050000B0
:104A20000C050000F7B5050000200C000193824240
:104A30005CD0161E402E00D940262F001C373800AF
:104A400000F0ECFBB1222B69D20080219C500122A6
:104A500089005A50A97E002901D11A621A600024E7
:104A6000731E2A69A34206D1019B002B03D0802329
:104A700002219B00D150012313621300FC33D9683B
:104A8000002902D1996A0029F9D0996A00290AD12E
:104A9000D960A323DB00D1583800C9B2013400F03B
:104AA000B2FBA642DCD8019A2B69002A04D11A0075
:104AB000FC32916A00290AD001210022AA765961AC
:104AC0001900FC3188680028FCD08A6007E00121C9
:104AD000A976D961D16C0029FCD00021D164FC33C6
:104AE0009A6A002A01D000229A62E0B2FEBD10B597
:104AF0000123FFF797FF10BD0300AC3310B504008E
:104B00001970643000F08AFB0123637610BD000049
:104B1000F8B500220D0001004276AC3103690400B3
:104B20000878B121C9005850802189005A500132BB
:104B30001A629A6026006436300000F081FB00287B
:104B40000ED03000276900F06DFB1E4BF850236932
:104B5000FC331A6A002A0CD19A6A002AF9D008E0BC
:104B60002369002D0AD11A00FC32916A002905D16F
:104B70000EE09A6A002AF3D11A62DBE701225A6139
:104B80001A00FC3291680029FCD00021916006E0F7
:104B90000121D961D16C0029FCD00021D1641A0017
:104BA0000020FC32916A81420BD0074990625A582A
:104BB00002305A50824204D0043A534253410230E8
:104BC000C01AF8BD1C050000C404000010B5012186
:104BD000FFF79EFF10BD000010B5132314220249F9
:104BE0000248FFF7D5FE10BD00400040B010002085
:104BF000F0B5474680B4CB0F98464A4C4B005B0D4E
:104C00001E1982B007000A00132E35DC002E57DB78
:104C1000454B040033411F000F4007430D00002F98
:104C200024D05B081C000C4020430027002807D03C
:104C3000132E00D172E08022D202324199430A43FE
:104C40004346DE00394B11009E1934687568380000
:104C500022002B0000F0C0FE009001910098019905
:104C600022002B0001F0E4F904000D0020002900CF
:104C700002B004BC9046F0BD332E0CDD802304004E
:104C80000D00DB009E42F1D102000B0000F0A4FEFB
:104C900004000D00EAE7264C0D00A44601246344FD
:104CA0006442DC40A446614604000142DED049086B
:104CB0000142C5D08027FF051F4188430743BFE756
:104CC0004B005B08034304000D00002BCED00B0308
:104CD0001B0B03435A42134380221B0B1203134046
:104CE0004A0C5204134319004346104ADB00D31800
:104CF0001C685D6822002B0000F06EFE00900191A0
:104D00000098019922002B0001F092F942464B00D5
:104D10005B08D607334304001D00A7E780273F0642
:104D200089E7C04601FCFFFFFFFF0F00D8880000A5
:104D3000EDFBFFFF03210A4802680A4302600948AD
:104D400002680A4302600849084A094B9B1A03DDBE
:104D5000043BC858D050FBDC00F0B4F9FBF70AFA6A
:104D60002405004054050040FC8A0000000000209B
:104D700020020020FEE7FEE7FEE7FEE7FEE7FEE793
:104D8000014B18607047C0465C010020F7B5002356
:104D9000202877D83C4B8000C258042A14D006D86B
:104DA000022A0DD00ED80423012A14D069E0062A65
:104DB0000ED00BD31A2A0DD002231B2A0BD060E091
:104DC000082308E0102306E0202304E0402302E04B
:104DD000802300E001232D4A1268082A04D9092AF9
:104DE00005D00A21022404E00821002401E011007A
:104DF0000124A02501261C272548ED004651254DFC
:104E0000254E2D681B02AD003D400195234D2D68B8
:104E100000958559AC466746214D3D401D4385515F
:104E20008359C0259C46009BAD021D40FF23674669
:104E30001B023B402B43019D1D43009B5F016023F0
:104E40001F402B003B431C4301238451154C03603E
:104E500063680F48002BFBD00024124B01255C60D7
:104E6000A123DB00C3584560A025ED0044511BB2CF
:104E7000914207D002D98A1AD34003E0521A9340D4
:104E800000E000231800FEBD5488000060010020EF
:104E9000007000405801002004050000540100206B
:104EA000FF00FFFFFC700040F0B520286CD8374BA6
:104EB0008000C258364B1E68002E2ED1C2243548C1
:104EC000A4000759344B03253B40C0273F023B4316
:104ED00003518023893C9B00FF3C03512F4F03600B
:104EE0002F4B803CD859FF3CA043D8510437D859A8
:104EF000A8432043D8510837D8590C35A843083D5A
:104F00002843D851A820C0001E508026C120760218
:104F100080001E501C601E4B1C600023142621487C
:104F200034005C43255804006F1C0FD114205843F3
:104F30002250A0200325C132FF329200C005155037
:104F4000194A08001268082A03D10BE0AA4218D1B6
:104F5000ECE7082A02D9083AD14002E00820821A78
:104F60009140080014225343E3189A680C495132C7
:104F7000FF32920058605050DA68C1239B00CA503B
:104F800002E00133032BCBD1F0BDC04654880000B2
:104F90006811002000E100E0FF00FFFF04050000B1
:104FA00000900040640100205C0100201E4BF0B521
:104FB000596C18001D4A002914D0A025A1260023F1
:104FC0000124ED05F600D1584F1C06D0D7187F6894
:104FD000002F02D027008F40AF5114333C2BF2D169
:104FE00000234364131DA025403294460020012471
:104FF0000F4EED05DA680F49920057180A4952180A
:10500000526C002A0CD01A1F1268511C05D0196866
:10501000FF2902D021009140A9513A00FC3250648E
:1050200014339C45E6D1F0BDFC90004064010020A3
:105030000C0500000090004000B5202816D80C4A4E
:1050400083009B58032911D8A0220800C133FF33E5
:10505000D2059B0000F014FB02080406002104E0C6
:105060000C2102E0042100E00321D15000BDC04624
:105070005488000020280DD8074B8000C058A0227B
:105080000123D2058340002901D1044901E0A12177
:10509000C90053507047C046548800000C050000FA
:1050A00003000020202B0AD8A222A021D200C9058B
:1050B0008858034A9B009B58D840012318407047EA
:1050C000548800002D4B10B51A78012A19D12C4AAA
:1050D0001268120715D12B4AE0241168F02208004B
:1050E000104021420BD128490968114209D12749B2
:1050F000274A11608021274A0902116001E0302807
:10510000F1D01A78012A0DD11D490968090709D182
:10511000F0201C4909680140402903D11A49096857
:10512000014223D01B68DBB2012B25D1144B1B6835
:105130001B0721D1134B1A68F0231A40A02A04D16F
:10514000114A12681A4203D016E0D02A14D1F7E7A8
:10515000114B1A68012A03D1C022104B1A600BE0D0
:105160000F4A1A601A68012AFCD1F5E7C121802094
:10517000C900C0054250D5E710BDC046E00F00F0A1
:10518000E40F00F0E80F00F0EC0F00F0DFFF07C0C5
:1051900004050040186C004000EC064014EC06408A
:1051A00075930000F7B506000D000C008B180193F5
:1051B000019B671B9C4207D0336821781B68300035
:1051C000984701340028F3D13800FEBD70B50500C2
:1051D0000C00081E07D001F089FF2B6802005B68F5
:1051E00021002800984770BD10B5FFF7EFFF10BDF4
:1051F00010B540220021040001F04BFB00232000E9
:105200002364636410BD3F23026C10B5541C23401B
:10521000446C9C4201D08154036410BD002303649C
:1052200043647047436C026C934206D03F21C25CDA
:1052300001330B404364100001E0012040427047FD
:10524000036C406C181A00D540307047436C026CF8
:10525000934201D0C05C01E0012040427047036CE2
:10526000406C5A1C3F231340181A42424241D0B2AC
:1052700070470120704710B503681322DB69984717
:1052800010BD70470369054A9950FC331A6A002A19
:10529000FCD0002201201A627047C0461C050000A5
:1052A000030010B55C331A781F231340012211004C
:1052B00099400D4B0424D967C221036989005C50D1
:1052C0005A60DA60A0220021D200995001220749D9
:1052D00052425A50064914305A500C395A5008312B
:1052E0005A50FFF79BFF10BD04E100E00C050000E1
:1052F0001405000010B51430FFF7A2FF10BD10B563
:105300001430FFF7A3FF10BD10B51430FFF78AFF6C
:1053100010BD0000030070B55E331C780269604B5D
:10532000D45003005D331C785E4BD45003006133CE
:105330001C785D4B012C0CD105005F352E78A22521
:10534000ED005651050060352E78A125ED0056512F
:1053500000E00024D4509623DB00994238D99623EC
:105360001B01994237D996235B01994236D996237E
:105370009B01994234D9E1239B01994232D996236A
:10538000DB01994231D9E123DB0199422FD99623E0
:105390001B0299422DD9E1231B0299422BD9962356
:1053A0005B02994229D9E1235B02994227D9E12383
:1053B0009B02994225D93D4B994224D9E123DB0236
:1053C000994223D9E1231B03994221D8384B21E08C
:1053D0009E23DB021EE09D231B031BE0354B19E0DF
:1053E000354B17E0EC239B0314E0344B12E0344BB5
:1053F00010E0344B0EE0344B0CE0344B0AE0344BFD
:1054000008E0344B06E08023DB0403E0324B01E08C
:1054100080235B0531490024535004232439535021
:105420001100FC31CC600C62C12101348900146090
:105430005C309460535003781F202200D9B208409A
:10544000824080342648FF345BB20251002B13DACD
:105450000F230B40083B234C9B089B001B19032484
:105460002140A140FC348C40DD69A543C0248C4020
:1054700021002943D96111E0194C9B089B001B199D
:1054800003242140A140C025FC348C40AD005E596E
:10549000A643C0248C40210031435951026070BDA5
:1054A0000C050000140500006C05000090D00300FE
:1054B00000D0BE0E00B013000050270000A04E0028
:1054C00000F0750000509D0000F0EB0000903A01E4
:1054D00000E0D70100B0AF0300705F0724050000B3
:1054E00000E100E000ED00E0F7B5009308AB1B78A9
:1054F00000250193FA2304009B0083600E4B456056
:105500000833036014300F001600FFF771FE23000C
:105510005C3327611E70009B084A9B00995823004A
:105520005D331970019B20009B009A5823005E3365
:10553000DD701A70FEBDC046E88800005488000087
:10554000036910B51A00FC32D2680400002A0AD0A0
:10555000A322D20099581430C9B2FFF754FE00229A
:105560002369FC33DA6010BD10B50248FFF7E8FF8D
:1055700010BDC0466C110020162307B5022200930F
:105580000249013B0248FFF7AFFF07BD0020004082
:105590006C1100207047000010B500F047F8FFF7CD
:1055A000F9FF012000F024F8FFF7EEF8FFF700F90B
:1055B000024B002BFAD000E000BFF7E7000000002C
:1055C000084A0949094B10B51B688858FA22190A7C
:1055D0001B0618439200002300F0D2F94904C00BC7
:1055E000084310BD0405000000100140D011002048
:1055F00070B5041E09D0FFF7E3FF050000F014F8B2
:10560000FFF7DEFF401B8442F8D870BD0022044B38
:105610009A60044A13680133DBB213607047C046D6
:10562000FC100140D011002070470000C421114A35
:1056300089005058104B0340C020000203435350D0
:10564000802391399B02FF39535013608023A3229A
:105650000021DB05D20099500122A1209A60074B5E
:10566000C0001950C120023180001950403019503B
:105670001A60704700E100E0FF00FFFF00100140EA
:1056800002B4714649084900095C49008E4402BCD5
:105690007047C046002243088B4274D303098B42F3
:1056A0005FD3030A8B4244D3030B8B4228D3030CF2
:1056B0008B420DD3FF22090212BA030C8B4202D394
:1056C0001212090265D0030B8B4219D300E0090ABC
:1056D000C30B8B4201D3CB03C01A5241830B8B42C5
:1056E00001D38B03C01A5241430B8B4201D34B03AE
:1056F000C01A5241030B8B4201D30B03C01A524113
:10570000C30A8B4201D3CB02C01A5241830A8B4297
:1057100001D38B02C01A5241430A8B4201D34B0280
:10572000C01A5241030A8B4201D30B02C01A5241E4
:10573000CDD2C3098B4201D3CB01C01A5241830998
:105740008B4201D38B01C01A524143098B4201D3D2
:105750004B01C01A524103098B4201D30B01C01AFD
:105760005241C3088B4201D3CB00C01A5241830877
:105770008B4201D38B00C01A524143088B4201D3A4
:105780004B00C01A5241411A00D201465241104604
:105790007047FFE701B5002000F0F0F802BDC046F9
:1057A0000029F7D076E7704703460B437FD40022E9
:1057B00043088B4274D303098B425FD3030A8B42A5
:1057C00044D3030B8B4228D3030C8B420DD3FF220F
:1057D000090212BA030C8B4202D31212090265D0DD
:1057E000030B8B4219D300E0090AC30B8B4201D390
:1057F000CB03C01A5241830B8B4201D38B03C01AD7
:105800005241430B8B4201D34B03C01A5241030B4D
:105810008B4201D30B03C01A5241C30A8B4201D3FE
:10582000CB02C01A5241830A8B4201D38B02C01AA9
:105830005241430A8B4201D34B02C01A5241030A20
:105840008B4201D30B02C01A5241CDD2C3098B4205
:1058500001D3CB01C01A524183098B4201D38B0182
:10586000C01A524143098B4201D34B01C01A524125
:1058700003098B4201D30B01C01A5241C3088B426A
:1058800001D3CB00C01A524183088B4201D38B0055
:10589000C01A524143088B4201D34B00C01A5241F7
:1058A000411A00D201465241104670475DE0CA0FCE
:1058B00000D04942031000D34042534000229C468E
:1058C00003098B422DD3030A8B4212D3FC22890198
:1058D00012BA030A8B420CD3890192118B4208D36E
:1058E000890192118B4204D389013AD0921100E0D0
:1058F0008909C3098B4201D3CB01C01A52418309E4
:105900008B4201D38B01C01A524143098B4201D310
:105910004B01C01A524103098B4201D30B01C01A3B
:105920005241C3088B4201D3CB00C01A52418308B5
:105930008B4201D38B00C01A5241D9D243088B420B
:1059400001D34B00C01A5241411A00D201466346AE
:1059500052415B10104601D34042002B00D5494212
:10596000704763465B1000D3404201B5002000F051
:1059700005F802BD0029F8D016E770477047C04609
:10598000F0B54F464646C0B41604360C994633006F
:1059900005042C0C070C150C63437E436F436543D1
:1059A0001C0CAD1964199C46A64203D980235B02E6
:1059B000984647446346250CEF191D044B464A435D
:1059C00043432D0C240464199918C91920000CBCF8
:1059D00090469946F0BDC046F8B556465F464D46DE
:1059E0004446F0B40F00FD0FAA4609037C002E00C8
:1059F0005F00450F490A7F0D2943C5001803BC46C7
:105A0000400A570F640DDB0F3843D2009A4500D18E
:105A1000AAE06646A61B002E00DCFFE06346002BD2
:105A200039D10300134300D0D9E06B0709D00F230D
:105A30002B40042B05D02B1DAB42AD416D424919C3
:105A40001D000B0200D482E0CA4B01349C4200D1FD
:105A5000FEE00A005646C84BED081A4050076405A0
:105A600052020543120B640D002112030B0D1B059E
:105A70006405120B1A436308C04CF60714401C431C
:105A8000640064083443280021003CBC90469946D9
:105A9000A246AB46F8BDB74B9C42C6D080231B0440
:105AA0001843382E00DDEBE01F2E00DD1EE1202321
:105AB0009B1B9C4603006746BB4098461300474625
:105AC000F3403B436746BA40571EBA4113430200B6
:105AD000F240EB1A9D42B6411D008A1A7642911B94
:105AE0000B0231D54A02560A002E00D1B4E0300034
:105AF00000F028FE0300083B1F2B00DDB5E020224C
:105B00002900D21AD1409E400A009D4032439C4257
:105B100000DDB1E01C1B631C1F2B00DDD5E0202144
:105B200014002800C91A8C40D8408D400443DA4044
:105B3000681E854111002543002476E74146314324
:105B400000D134E2310045466B0700D06FE756467E
:105B50004807ED08C9080543864B9C4235D00A0327
:105B60006405120B640D7FE76346E31A9B46002B26
:105B700000DC8BE06746002F3CD07E4FBC4200D15A
:105B800053E780273F0438435B46382B00DCF7E0BF
:105B90000243501E82410020D2B253194218AB4238
:105BA00089411D00494289180B02CDD5714B013442
:105BB0009C4200D13DE101206F4A6B080A40284019
:105BC0001843D507054351082FE72B000B4300D19D
:105BD000CBE180231B030B431A03120B44E7013E66
:105BE000002E6DD1AE1AB5429B41091A5B42C91A0B
:105BF000350075E70700174300D116E701235B4224
:105C00009C46E3445B46002B00D0E0E0AA18AA4281
:105C10009B4109185B4259181500C5E7002E75D144
:105C2000661C7605760D012E00DCF3E0AE1AB04658
:105C30004545BF410E1A7F42F61B370200D48FE064
:105C4000551BAA42B641411A76428E1B9A464BE733
:105C500056460022002507E7280000F073FD20309B
:105C60000300083B1F2B00DC49E72A00283882404C
:105C700000259C4200DC4DE73F49E41A1140D4E680
:105C80000243501E8241D3B2002222E7002B00D0F3
:105C9000F3E0631C9C465B055B0D012B00DC9FE081
:105CA000344B9C4500D1C3E0AA180918AA42804190
:105CB00040424118CD075208154349086446B4E6EE
:105CC0002C4B9C4200D0ECE6AFE611001F3CE140BB
:105CD0000C00202B00D17FE04021CB1A9A401543C5
:105CE0006A1E95410021254300242DE7330007005B
:105CF000203BDF403B00202E70D04027BE1BB04031
:105D00000243501E824113430022E2E6002C4FD092
:105D1000184CA44500D1ABE08024240476422143F2
:105D2000382E00DDDFE01F2E00DD43E12027BC1B05
:105D3000A1460C004F46BC40A0462C004746F4400C
:105D40003C434F46BD406F1EBD41F1402C43151BE7
:105D5000AA429241411A5242891A64469A46BFE6C3
:105D600041464546314300D0BEE6002600240025CA
:105D7000F2E6C046FF070000FFFF7FFFFFFF0F8036
:105D80001F2B59DC2027FF1ABC46070063469F40A3
:105D90005B46B9461700DF40B8464F4643461F43AF
:105DA00063469A40531E9A415B463A43D840F4E614
:105DB0000C002C435CD0F643002E55D1551BAA4253
:105DC000A441411A6442091B9A46644688E6964FEC
:105DD000BC4200D0D8E628E6002280E700208FE70A
:105DE0000B002B43002C00D0C2E0002B00D101E1BE
:105DF0000300134300D118E6AB18AB42B6410918B3
:105E0000764271180A0200D409E1884A1D00114047
:105E100064460AE6002C5BD10E002E4300D08AE0D7
:105E20000100114300D1C2E0010015009A46FCE5D3
:105E30006446002100258FE620235B429C46DC441B
:105E400063460700DF405B46BC46202B00D1ACE038
:105E500040235F46DB1B98400243501E824163464D
:105E600013431A00002098E66F4CA44500D057E772
:105E70000100150064469A46D7E5002C39D10C0084
:105E80002C436ED0DB43002B1AD0674CA44568D05E
:105E9000382B00DDA4E01F2B00DDAEE020240F0036
:105EA000E41AA740B9462F00DF40B846A3464F4644
:105EB000444627435C46A5406C1EA541D9403D435E
:105EC000AD1895429B4109185B42591864466BE630
:105ED0000C002C4315D1010011437BD001001500AB
:105EE0009A46514CA1E50D43691E8D410021ECB24B
:105EF0002DE74D4CA44534D0802424045B4221433B
:105F0000C6E7040014434ED0ED084C072C4380250F
:105F1000C9082D03294208D0C6082E4205D1D2084F
:105F2000410711430C009A463100620FC900E50099
:105F300011433D4C79E50600164300D175E5AE1AD4
:105F4000B0464545BF410E1A7F42F61B370200D4CA
:105F5000F4E5551BAA42B641411A7642891B9A467E
:105F600063E50100150064465FE5002200257BE53E
:105F7000002B3BD00300134315D0ED084B072B43F8
:105F80008025C9082D03294207D0C4082C4204D11A
:105F900041070B002100D2081343C9005A0F1143D7
:105FA000DD00214C41E5204C3FE5002054E7002670
:105FB0000025D1E534000F00203CE7403C00202EB6
:105FC0002BD04027BE1BB1400D43691E8D410021DF
:105FD0002C43BCE6802100260903134C0025BBE5B9
:105FE0000D43691E8D410021EDB269E701001500E6
:105FF0000D4C1AE50100150017E51C000F00203CB0
:10600000E7403C00202B0CD04027FB1A99400D4361
:10601000691E8D410021254352E70021D4E71D0070
:1060200092E50021F3E7C046FF070000FFFF7FFF76
:10603000F0B557464E464546E0B40E001100F20F4B
:106040009246C500420F180337037400400A4E0FF2
:106050007F0A3043CF4E17435A00640D520DDB0FB9
:10606000C900B24200D1E5E001267340A61AB44649
:10607000534500D1AFE0002E00DC0DE1002A3AD1FB
:1060800003000B4300D0E4E06B0709D00F232B4043
:10609000042B05D02B1DAB42AD416D427F191D0075
:1060A0003B0200D488E0BB4B01349C4200D110E19C
:1060B0003A00B94B51461A4001235007ED085202ED
:1060C00064050543120B640D0B40002128001203E8
:1060D0000D0D120B64052D0515436208AF4CDB074F
:1060E0002C401443640064081C4321001CBC9046EF
:1060F0009946A246F0BDA74B9C42C5D080231B0405
:1061000018436346382B00DDFDE01F2B00DD30E136
:10611000624620239B1A02009A40664690460A0077
:106120009940F24046464B1E994132431143634623
:106130000200DA40691A8D429B410D00BA1A5B4297
:10614000D71A3B0235D57A02530A98464346002BAC
:1061500000D1C4E0404600F0F5FA0300083B1F2BD5
:1061600000DDC5E020222900D21A4746D1409F40D9
:106170000A009D403A439C4200DDC0E01C1B631CAA
:106180001F2B00DDE4E0202114002800C91AD840AC
:106190008C408D400443DA40681E8541170025433A
:1061A000002471E7424663461A4300D14CE2674639
:1061B00045466B0700D069E7012351467807ED0893
:1061C000FA080B40054373498C4238D0120364052A
:1061D000120B640D79E7002E00DC9AE0002A47D00C
:1061E0006C4A944200D14FE7802212041043624669
:1061F000382A00DC08E10143481E81410022C9B26F
:106200004919D219A942BF410D007F42BF183A0275
:1062100000D442E15F4A0134944200D14EE10120B2
:106220005D4A69083A4028400843D50705435708A6
:106230009A4629E706000E4300D017E714E7290025
:10624000114300D1F9E1802109030A431203120B23
:106250003BE701235B429846C4446346002B72D15E
:10626000691A8D429B413F1A5B42FF1A0D0068E795
:1062700002000A4300D107E7012252429046C4447B
:106280006246002A00D0E6E06918A942B6413F18EC
:106290007642F7190D00BAE7002E00D080E0621CAC
:1062A0005205520D012A00DCF9E06A1A91464D456B
:1062B000B6413A1A7642921B9046120200D499E0F7
:1062C0004D1BA9428941C71B49427A1A90469A46FA
:1062D0003CE752460123002513400022F5E6280042
:1062E00000F030FA20300300083B1F2B00DC39E7B8
:1062F0002A002838824000259C4200DC3EE7264FD9
:10630000E41A1740C0E60143481E81410022C9B289
:1063100010E7002E00D0F1E0621C94465205520DA9
:10632000012A00DCA0E01B4A944500D1C5E06918B1
:10633000A94292413F185242D2194908D5070D434C
:1063400057086446A0E6134B9C4200D0D9E69BE672
:1063500011001F3CE1400C00202B00D180E04021C7
:10636000CB1A9A4015436A1E954100272543002405
:106370001FE763460200203BDA406346202B71D0C2
:10638000402366469B1B98400143481E81411143B0
:106390000022CFE6FF070000FFFF7FFFFFFF0F8017
:1063A000002C48D0CA4CA24200D1A2E07442A146BF
:1063B0008024240427434C46382C00DDDBE01F2CCE
:1063C00000DD44E14E462024A41B3E00A640A24628
:1063D000B0464C462E00E640B44646466446264348
:1063E0005446A5406C1EA54134002C434D46EF4059
:1063F0000D1B28E04A4643464D461A4300D0A5E609
:10640000002300240025DEE61F2A5ADC66462022EF
:10641000921B060096409146B04662460E00D6405A
:10642000424616434A4691404A1E91410200604648
:106430003143C240E4E63C002C435AD0F443A14629
:10644000002C52D14D1BA9428941C71B49427F1ADA
:1064500014009A4675E69E4A944200D0C7E613E6B9
:1064600000227FE700208FE7002C00D0C8E03B002F
:106470002B4300D10FE103000B4300D104E6691860
:10648000A9429B413F185B42DF193B0200D41AE14D
:10649000904B0D001F406446F6E59A4689E63A00A7
:1064A0002A43002C5CD1002A75D102000A4300D196
:1064B000CAE007000D009A46E6E564460022002582
:1064C00081E662460600203AD6406246B046202A5F
:1064D00000D1B7E040226646921B904001434246FD
:1064E000481E8141114300228AE6794CA24200D025
:1064F00061E707000D0014009A46C5E5002C41D164
:106500003C002C4378D0F443A146002C20D0704CA2
:10651000A24271D04C46382C00DDB2E01F2C00DDC9
:10652000BCE02026341BA2463C005646B4404E46F2
:10653000A0462C00F440A446444666463443A44694
:106540005446A54064466E1EB54125434C46E7407F
:106550006D188D4289413F184942CF19140056E603
:10656000002A2FD102000A4300D184E007000D0069
:106570009A46574C88E53D436F1EBD41ECB200275B
:106580000D1B60E7524CA24236D07442802636047E
:10659000A1463743BEE702000A4300D174E56A1AF8
:1065A00090464545B6413A1A7642921B94461202ED
:1065B00000D4F7E54D1BA9428941C71B49427F1A08
:1065C0009A4661E502000A433AD0ED087C072C4365
:1065D0008025FA082D032A4208D0C7082F4205D18A
:1065E00045072C003A009A46C9080C43670FD200B1
:1065F000E5001743364C47E507000D00140043E55E
:106600003A002A4343D002000A4319D0ED087C0720
:106610002C438025FA082D032A4207D0C6082E42B3
:1066200004D147073C003200C9080C43D700620F71
:10663000E50017439A46264C26E50022002544E54E
:10664000234C21E5002049E700230025BBE54C460B
:106650003E00203CE6404C46B446202C31D040243D
:106660004E46A61BB7403D436C1EA54164462C43D5
:1066700000270D1BE7E6802200231203144C00259F
:10668000A1E53D436F1EBD410027EDB260E7070065
:106690000D000F4CF8E407000D00F5E44E463C00F9
:1066A000203EF440A0464C46202C0ED040244E46BE
:1066B000A41BA7403D436F1EBD4144460027254310
:1066C00046E70027CFE70D0073E50027F2E7C04655
:1066D000FF070000FFFF7FFF0B0330B5134D1A0BC0
:1066E0004B005B0DC90F0024AB4211DD104CA342DF
:1066F00010DC8024640322430E4CE41A1F2C0CDDB2
:106700000D48C31ADA4013005C42002900D11C0076
:10671000200030BD094BCC18FAE7E040084CA446F5
:1067200063449A4013000343EEE7C046FE030000B3
:106730001D0400003304000013040000FFFFFF7F6E
:10674000EDFBFFFF1C2101231B04984201D3000C29
:1067500010391B0A984201D3000A08391B099842D4
:1067600001D30009043902A2105C40187047C046EA
:10677000040302020101010100000000000000000A
:106780007FB51D000A4B06001B68D868002A02D19D
:10679000084C230001E01300074C029300913300E2
:1067A0002A000649019400F021F800F023FEC046BB
:1067B000000200206C81000018890000258900007B
:1067C000084B10B50400002B02D0002100E000BFF0
:1067D000054B1868836A002B00D09847200001F011
:1067E000F3FAC04600000000588900000EB403B55B
:1067F000010003AB044804CB0068019300F016F9D4
:1068000002B008BC03B01847000200200E4B70B560
:1068100000251E000D4CE41AA410A54204D0AB00C4
:10682000F35898470135F8E701F0D0FA084B0025F6
:106830001E00084CE41AA410A54204D0AB00F35883
:1068400098470135F8E770BD0802002008020020D3
:10685000080200201802002010B5034B0100186840
:1068600000F066F810BDC0460002002010B5034BD2
:106870000100186800F016F810BDC04600020020A4
:10688000002310B59A4203D0CC5CC4540133F9E71D
:1068900010BD03008218934202D019700133FAE749
:1068A0007047000030B500293ED004390B68002B3A
:1068B00000DAC9181D4A13681400002B02D14B607E
:1068C000116031E08B420DD90A688818834203D1E8
:1068D00018685B6882180A604B60216024E08A4275
:1068E00003D813005A68002AF9D11D685C198C423C
:1068F0000BD10968691858181960824214D11068C0
:106900005268411819605A600EE08C4202D90C237B
:10691000036009E008680C18A24203D114685268A9
:10692000201808604A60596030BDC046D811002068
:10693000032370B5CD1C9D43083506000C2D01D2F4
:106940000C2505E0002D03DA0C230020336040E025
:10695000A942F9D81F4B1C681A002100002913D046
:106960000B685B1B0DD40B2B02D90B60CC181EE0FF
:106970008C4202D1636813601AE04B6863600C00BC
:1069800016E00C004968E9E7134C2368002B03D19B
:10699000300000F033FB20602900300000F02EFBB7
:1069A000431CD1D00323C41C9C43A0420AD12560C0
:1069B000200007220B30231D9043C31A09D05A42EE
:1069C000E25006E0211A300000F018FB431CEED123
:1069D000BAE770BDD8110020D4110020936810B51B
:1069E000013B9360002B05DA9469A34208DBCBB22C
:1069F0000A2B05D01368581C10601970C8B201E04A
:106A000000F02CFC10BDF8B506000F001400D518DE
:106A1000AC4208D021783A003000FFF7DFFF0134A4
:106A2000431CF5D100E00020F8BD0000F0B59FB098
:106A300006000F0002920593002804D08369002B02
:106A400001D100F0D3FD7F4B9F4201D1776808E070
:106A50007D4B9F4201D1B76803E07C4B9F4200D140
:106A6000F768BB891B070AD53B69002B07D00023B9
:106A700006AD6B6120336B761033AB763DE03900A9
:106A8000300000F043FC0028F1D001204042D6E065
:106A9000059A111D12680591002A00DA7FE009921B
:106AA000013423782E2B00D18DE021780322684811
:106AB00000F082FE002807D0654B2A68C01A4023E8
:106AC000834013432B6001342178631C0622614804
:106AD0000293297600F070FE002800D19DE05E4B05
:106AE000002B00D090E00722059B07339343083327
:106AF00005936B69039A9B186B61029C2378002BAA
:106B000004D1029BE31A049312D003E0252BF8D0A2
:106B10000134F3E7049B029A39003000FFF773FF5A
:106B2000431C00D186E06A69049B944663446B6110
:106B30002378002B7ED00122002352426A6002A9F2
:106B40005432521801342B60EB60AB601370AB65AC
:106B500021780522414800F02FFE002808D03F4B45
:106B60002A68C01A0123834013432B600134EFE7E6
:106B70002B68DA0604D55322202102A812181170BE
:106B80001A0704D553222B2102A81218117022785B
:106B90002A2A00D17CE7099B00200A2105E0524205
:106BA000EA60022213432B607AE72278303A092AFE
:106BB00004D84B4301349B180120F6E7002800D18C
:106BC0006FE709936DE763782A2B0AD1059B02349E
:106BD0001A1D1B680592002B01DA01235B42079303
:106BE00063E700230A201A0001346B6021783039F2
:106BF000092904D84243013452180123F6E7002B37
:106C000000D152E7079250E705AB00933A00144BCE
:106C10002900300000E000BF07E005AB00933A0018
:106C20000F4B2900300000F08BF80390039B0133D9
:106C300000D05EE7BB895B0600D526E70B981FB046
:106C4000F0BDC046908A0000B08A0000D08A0000E3
:106C50006289000066890000000000005C89000075
:106C6000076A0000F7B5170001938A680B69009066
:106C70000C00934200DA130022003B60433212788A
:106C8000002A01D001333B6023689B0602D53B6894
:106C900002333B60062523681D401ED0230043338A
:106CA0001B785A1E9341226892061CD53020E118A9
:106CB0004331087021005A1C45310978A21843322B
:106CC000023311700FE0220001231932019900985C
:106CD000089EB047431C0ED00135E3683A689B1A02
:106CE0009D42F0DBDAE72200019943320098089DCB
:106CF000A847431C02D10120404220E0062320681F
:106D0000E1683A6803400025042B03D18D1AEB4358
:106D1000DB171D40A3682269934201DD9B1AED1821
:106D20000027BD420AD0220001231A32019900989F
:106D3000089EB047431CDED00137F2E70020FEBDBD
:106D4000F0B58BB006920A00433207930590049287
:106D50000A7E0C00109B6E2A00D1ABE011D8632A8A
:106D600022D009D8002A00D1B5E0582A00D0C5E0C9
:106D700045310A70814A4FE0642A1DD0692A1BD030
:106D8000BCE0732A00D1AAE009D86F2A29D0702A62
:106D900000D0B3E0202209680A43226037E0752A58
:106DA0001FD0782A33D0A9E00E001A684236111D90
:106DB000196013683370A4E021681A68080606D4C5
:106DC000490604D5111D19600023D55E02E0111D8E
:106DD00019601568002D3BDA2D23049A6D4213705B
:106DE00036E021681A68080606D4490604D51568F5
:106DF000111D1960ADB202E0111D196015685F4BDD
:106E0000227E039308276F2A1DD00A271BE0220049
:106E10007821453211705A4A19680392081D226878
:106E200018600D68100602D4500600D5ADB2D30725
:106E300002D520231A4322601027002D03D12023DE
:106E400022689A4322602300002243331A7002E032
:106E50000A274A4B03936368A360002B09DB0422D3
:106E6000216891432160002D05D1049E002B11D093
:106E70007BE0002D79D0049E28003900FEF790FCBD
:106E8000039B013E5B5C280033703900FEF702FC77
:106E9000051EF1D1082F09D12368DB0706D56368E9
:106EA0002269934202DC3023013E3370049B9B1B1A
:106EB00023612BE009681A68080607D4490605D53E
:106EC000111D19601368A28A1A8004E0111D19604F
:106ED000136862691A600023049E236116E01A6831
:106EE000111D1960166800216268300000F064FC12
:106EF000002801D0801B6060636803E026004236F2
:106F00003270012323610023049A1370079B09AA9E
:106F100000932100069B0598FFF7A4FE431C02D1B5
:106F20000120404227E02369320006990598079D19
:106F3000A847431CF4D0236800259B070FD4099B66
:106F4000E068984217DA180015E022000123193290
:106F500006990598079EB047431CE1D00135E368C8
:106F6000099A9B1A9D42F0DBE9E72600039B423613
:106F70001B7833708EE70BB0F0BDC0466D89000002
:106F80007E890000154B10B51C68A36B002B15D132
:106F90001820FFF761FC124BA0630380114B012204
:106FA0004380114B8380114BC380114B0381052318
:106FB000438106338381002302614361A46B0D4A40
:106FC000206961690C4BFEF7DBFC0122002380186D
:106FD0005941206161614800400810BD0002002055
:106FE0000E330000CDABFFFF341200006DE6FFFF53
:106FF000ECDEFFFF2D7F954C2DF45158002370B52A
:10700000064C05000800236000F0C8FE431C03D1B5
:107010002368002B00D02B6070BDC046CC2400201C
:107020000CB430B5164B9DB00C1E1D6804DA8B23D2
:1070300001202B6040421DE0822302A99B008B812E
:107040000023029008619C4200D0631E8B604B615C
:1070500001235B42CB81209A21AB2800019300F0F1
:1070600053FC431C01DA8B232B60002C02D000233D
:10707000029A13701DB030BC08BC02B01847C0465D
:10708000000200200EB410B59DB002A90290086164
:107090000B48822488604861012040421FABC881B0
:1070A000084804CBA400006801938C8100F02CFCFC
:1070B0000023029A13701DB010BC08BC03B018471F
:1070C000FFFFFF7F0002002002780B78002A03D028
:1070D000013001319A42F7D0D01A7047031C0A7868
:1070E00001311A700133002AF9D170470023C25CC4
:1070F0000133002AFBD1581E7047030030B5002A27
:107100000DD00C7801335D1E013A2C700131002C3A
:10711000F5D19A189A4202D01C700133FAE730BDBB
:10712000F0B51E00454B87B01B6801920293082200
:107130000B00059003911C7802995D1C0919487891
:10714000104001D02B00F6E72D2C04D19D1C5C785B
:107150000123009304E000902B2C01D15C789D1C4E
:10716000002E02D0102E0AD162E0302C5ED12022F7
:107170002B789343582B54D110266C780235009FFE
:1071800031007B1E9F412E4BFF183800FEF708FB95
:10719000380004913100FEF77DFA00230322070036
:1071A00094461800029A121951780422114201D013
:1071B000303C07E06246114017D03722012900D049
:1071C0002032A41AA64210DD5A1C0BD0B84207D8B0
:1071D00002D1049B9C4203DC70430123201801E090
:1071E00001235B422C780135DCE75A1C0BD1009857
:1071F000059A431E9841124BC01822231360019B2D
:10720000002B0AD117E0009A002A00D04042019AD0
:10721000002A10D0039A002B00D06A1E019B1A602E
:1072200009E03024002EAAD10826A8E70A26A6E7FE
:10723000302C9CD0A3E707B0F0BDC046040200206C
:10724000FFFFFF7F10B513000A000100024800682D
:10725000FFF766FF10BDC04600020020F8B505002C
:107260000F001400002804D08369002B01D100F026
:10727000BDF9234B9C4201D16C6808E0214B9C4234
:1072800001D1AC6803E0204B9C4200D1EC68A369BB
:10729000A360A3891B070AD52369002B07D02368A5
:1072A0002269FEB2981A636998420FDB08E0210058
:1072B000280000F02BF80028F1D0012040421DE00A
:1072C0002100280000F024F90028F6D1A36801303D
:1072D000013BA36023685A1C22601F7063699842B7
:1072E00005D0A3893000DB0708D50A2E06D121007E
:1072F000280000F00DF90028DFD13000F8BDC046AD
:10730000908A0000B08A0000D08A0000354B70B52A
:107310001D6806000C00002D05D0AB69002B02D1C2
:10732000280000F063F9304B9C4201D16C6808E002
:107330002E4B9C4201D1AC6803E02D4B9C4200D106
:10734000EC68A3899AB2110723D4D10607D4092285
:107350000120326037321343A381404240E053079B
:1073600013D5616B002908D023004433994202D021
:107370003000FFF797FA002363632422A389934325
:10738000A38100236360236923600822A389134338
:10739000A3812369002B0BD1A023A2899B0013405A
:1073A00080229200934203D02100300000F0B2F915
:1073B0000123A289134005D00023A36063695B42C7
:1073C000A36103E0910700D46369A36000202369EF
:1073D000834205D1130603D540231A43A281013805
:1073E00070BDC04600020020908A0000B08A0000F4
:1073F000D08A000010B5062000F0AEFB012000F09E
:10740000E3FC0000F7B58A8905000C0013075AD485
:107410004B68002B02DC0B6C002B19DDE76A002F98
:1074200016D000232E682B6080235B011A4001D008
:10743000606D14E00123216A2800B847431C0ED177
:107440002B68002B0BD01D2B01D0162B02D12E60E8
:1074500000205AE04022A3891343A38155E0A38969
:107460005B0706D56368C01A636B002B01D0236CE1
:10747000C01A00230200216A2800E76AB847A389DE
:10748000421C06D129681D293AD8204ACA40D20791
:1074900036D50022626022692260DB0405D5431CD8
:1074A00002D12B68002B00D16065616B2E60002932
:1074B000CED023004433994202D02800FFF7F2F9DE
:1074C0000020606321E00F69002FC1D00B680F60BE
:1074D000DB1B01930023920700D14B69A36003E0FB
:1074E000019B3F181B1A0193019B002BB0DD019BF0
:1074F0003A00216A2800A66AB0470028F0DCA38978
:10750000402201201343A3814042FEBD01004020E0
:107510000B6970B505000C00002B01D100201CE0A8
:10752000002804D08369002B01D100F05FF80B4BD9
:107530009C4201D16C6808E0094B9C4201D1AC68C7
:1075400003E0084B9C4200D1EC680C22A35E002BA8
:10755000E4D021002800FFF755FF70BD908A00009D
:10756000B08A0000D08A000010B5024900F0B0F8DF
:1075700010BDC04611750000002310B50400036063
:107580004360836081814366C2810361436183619B
:10759000190008225C30FFF77CF9054B2462636216
:1075A000044BA362044BE362044B236310BDC0464B
:1075B000997B0000C17B0000F97B0000257C000066
:1075C00070B568254B1E5D430E0029007431FFF72E
:1075D000AFF9041E08D000212A00016046600C307B
:1075E000A0606832FFF755F9200070BD836913B5BC
:1075F0000400002B28D18364C3640365134B144A31
:107600001B6882620193984201D1012383612000AB
:1076100000F020F86060200000F01CF8A06020005E
:1076200000F018F80022E06004216068FFF7A4FF72
:1076300001220921A068FFF79FFF02221221E068C2
:10764000FFF79AFF0123A36113BDC04658890000CC
:1076500069750000F8B51D4B06001D68AB69002B6D
:1076600002D12800FFF7C2FF4835AC686B68013BC8
:1076700005D40C22A75E002F10D06834F7E72B68E2
:10768000002B01D02D68F0E704213000FFF798FFB0
:1076900028600028F6D10C23336016E00123200077
:1076A0005B42E3810233A38167662760A76067605E
:1076B00027616761A7615C3008223900FFF7E9F8AC
:1076C00020006763A763A764E764F8BD58890000DA
:1076D000F7B504000700002601914834002C16D0AD
:1076E0006368A5680093009B013B00930DD4AB89B0
:1076F000012B08D90E22AB5E013304D029003800DB
:10770000019B984706436835EDE72468E6E73000BB
:10771000FEBD0000F0B58B8991B006000C009B0700
:1077200026D40E23C95E002904DA8023A5891D40D2
:1077300010D10CE001AA00F0A1FA0028F5DBF0233B
:10774000029D1B021D401A4BED186B425D418027C4
:10775000FF0001E00025402739003000FFF7E8F87E
:1077600000280CD1A3899A051FD402221343A381B8
:1077700023004733236023610123636115E08022E6
:107780000C4BB362A38920601343A381206167611E
:10779000002D0AD00E23E15E300000F081FA0028AF
:1077A00003D00122A3891343A38111B0F0BDC046C9
:1077B00000E0FFFF69750000C9B28218904204D052
:1077C00003788B4202D00130F8E70020704710B5F3
:1077D000884202D98B18984201D3002305E09B1AF6
:1077E000013A08D3995C8154FAE7934203D0CC5C08
:1077F000C4540133F9E710BDF8B506000C001500BC
:10780000002904D11100FFF793F8040018E0002AC2
:1078100003D1FFF747F82C0012E000F067FA854229
:107820000ED929003000FFF783F8071E07D021008A
:107830002A00FFF725F821003000FFF733F83C005D
:107840002000F8BDF0B58E6885B007000C000392EB
:1078500001939E4243D890238A89DB001A423ED08E
:1078600003250969236801985B1A029363695D43E4
:10787000EB0F5D19029B6D1001331B18AB4200D951
:107880001D00530510D529003800FFF751F8061EDA
:1078900014D0029A2169FEF7F3FFA289194B134015
:1078A00080221343A38112E02A003800FFF7A4FFCF
:1078B000061E0CD121693800FEF7F4FF0C2340228C
:1078C00001203B60A38940421343A38117E0029B40
:1078D0002661F61826606561019EED1AA560019B80
:1078E000B34200D21E00320003992068FFF76FFFF9
:1078F0000020A3689B1BA36023689E19266005B027
:10790000F0BDC0467FFBFFFFF0B59FB0029005932E
:107910008B890F0016001B0610D50B69002B0DD1AB
:107920004021FFF705F838603861002804D10C23A6
:10793000029A01381360D8E040237B61002306AD32
:107940006B6120336B761033AB7634002378002BD9
:1079500003D1A31B049312D003E0252BF9D00134EB
:10796000F4E7A31B320039000298FFF76BFF431CBA
:1079700000D1B4E06A69049B944663446B61237848
:10798000002B00D1ABE00122002352426A6002A921
:107990005432521801342B60EB60AB601370AB654E
:1079A000534E217805223000FFF706FF002807D04C
:1079B0000123801B83402A68013413432B60EFE7C7
:1079C0002B68DA0604D55322202102A81218117060
:1079D0001A0704D553222B2102A8121811702278FD
:1079E0002A2A03D0099B00200A210EE0059A111DC6
:1079F00012680591002A01DB099204E05242EA6014
:107A0000022213432B6001340BE02278303A092A1A
:107A100004D84B4301349B180120F6E7002800D01E
:107A2000099323782E2B1ED163782A2B0AD1059B2C
:107A300002341A1D1B680592002B01DA01235B42F8
:107A4000079310E000230A201A0001346B602178AC
:107A50003039092904D84243013452180123F6E78A
:107A6000002B00D00792234E217803223000FFF72D
:107A7000A3FE002806D04023801B83402A680134DF
:107A800013432B60217806221B48661C2976FFF7DA
:107A900093FE002812D0194B002B06D10722059B1C
:107AA000073393430833059314E005AB00933A0082
:107AB000134B2900029800E000BF07E005AB0093DC
:107AC0003A000F4B29000298FFF73AF90390039B05
:107AD000013304D06B69039A9B186B6135E7BB894E
:107AE0000B985B0601D5012040421FB0F0BDC04697
:107AF0005C890000628900006689000000000000C7
:107B00004578000070B504000D1E1F2D04D9162302
:107B10000360012040421EE0426C002A04D08B002A
:107B2000D2181368002B08D1200000F031F82A0089
:107B30000100200000F01AF80DE00020012B0AD00F
:107B4000591C03D117332360013004E000242800BE
:107B500014609847200070BD10B5034B01001868F1
:107B6000FFF7D0FF10BDC04600020020002370B513
:107B7000064C050008001100236000F0F7F8431CD4
:107B800003D12368002B00D02B6070BDCC240020D3
:107B900010B500F0DBF810BD70B50C000E25495F84
:107BA00000F0B0F8002803DB636D1B18636503E089
:107BB000A289024B1340A38170BDC046FFEFFFFFB7
:107BC000F8B51F008B8905000C001600DB0505D5F4
:107BD0000E23C95E0022022300F074F8A289054B2F
:107BE00028001340A38132000E23E15E3B0000F029
:107BF0001FF8F8BDFFEFFFFF70B50C000E25495FC1
:107C000000F060F8A389421C03D1054A1340A38108
:107C100004E0802252011343A381606570BDC04619
:107C2000FFEFFFFF10B50E23C95E00F015F810BD81
:107C300070B50500080011000022064C22601A00F1
:107C400000F0BAF8431C03D12368002B00D02B604E
:107C500070BDC046CC240020002370B5064C050042
:107C60000800236000F062F8431C03D12368002B56
:107C700000D02B6070BDC046CC240020002370B51E
:107C8000064C050008001100236000F057F8431C63
:107C900003D12368002B00D02B6070BDCC240020C2
:107CA000002370B5064C05000800236000F056F86C
:107CB000431C03D12368002B00D02B6070BDC0464D
:107CC000CC24002070B50500080011000022064CED
:107CD00022601A0000F052F8431C03D12368002BE5
:107CE00000D02B6070BDC046CC2400200B1F1A684A
:107CF000101F002A04DA891804390B68D0180438D8
:107D00007047000070B50500080011000022064C05
:107D100022601A0000F03AF8431C03D12368002BBC
:107D200000D02B6070BDC046CC240020582201201A
:107D3000014B40421A607047CC2400205822012099
:107D4000014B40421A607047CC2400205822012089
:107D5000014B40421A607047CC2400205822024B4D
:107D600000201A607047C046CC2400205822012011
:107D7000014B40421A607047CC2400205822012059
:107D8000014B40421A607047CC2400205822012049
:107D9000014B40421A607047CC240020044A13680B
:107DA000002B03D01818106018007047014BF9E73A
:107DB000DC110020D024002058220120014B404239
:107DC0001A607047CC240020FEE7C046F8B5C046D4
:107DD000F8BC08BC9E467047F8B5C046F8BC08BC65
:107DE0009E467047F6060000880600000607000061
:107DF0003C07000078070000B2070000EE07000013
:107E000016080000540800009A080000F608000058
:107E10003A090000A0090000EC090000140A000063
:107E20004E0A0000980A0000C00A0000F80A00008C
:107E3000300B00006C0B0000F20B0000BA0C0000CD
:107E4000480D0000A60D0000E80D00000A0E00001D
:107E5000120E0000F40E0000F6060000F606000008
:107E6000F6060000F6060000400F0000AA0F000012
:107E7000141000005E100000C01000004611000049
:107E8000CE1100001C12000066120000AC120000AF
:107E9000F81200004413000090130000DE130000ED
:107EA0003414000072140000DE1400000E150000EF
:107EB0005A150000A6150000F21500002C1600004F
:107EC00078160000F6060000F6060000F606000030
:107ED000F6060000C4160000F41600002417000087
:107EE0005017000080170000AC170000F6060000D5
:107EF000F6060000F6060000F6060000E417000093
:107F00002C18000078180000A8180000D4180000F1
:107F1000021900004C190000F6060000F6060000E9
:107F2000F60600007A190000AA190000DA1900000C
:107F30000A1A0000361A0000661A0000921A0000A1
:107F4000BC1A0000E61A0000161B0000461B0000C9
:107F5000881B0000B41B0000E41B0000101C000084
:107F6000F6060000F6060000F6060000F606000021
:107F7000F6060000401C00006C1C0000981C00006D
:107F8000C41C0000F01C0000281D0000601D000043
:107F9000981D0000D01D0000FC1D00002A1E0000DE
:107FA0005A1E0000F6060000F6060000F606000065
:107FB000F6060000F6060000F6060000F6060000D1
:107FC000F6060000F6060000F6060000F6060000C1
:107FD000F6060000F6060000F6060000881E000007
:107FE000B61E000066616C73650074727565006C86
:107FF000697374206F66202564206974656D730051
:108000006F626A656374206F6620636C6173733A94
:1080100020256400537461636B20756E646572661D
:108020006C6F77000D0A564D2050616E69633A20DF
:1080300025730D0A00496E73756666696369656E1E
:1080400074206D656D6F727920666F72204D696363
:10805000726F426C6F636B73206F626A656374202A
:108060006865617000496E73756666696369656EFF
:1080700074206D656D6F727920666F72204D696333
:10808000726F426C6F636B7320737461636B006219
:108090006164206F626A65637420617420256C647A
:1080A0000A0025783A20256420776F7264732C20AB
:1080B000636C61737349442025640A0048656164F8
:1080C00065723A2025780A0009307825782C0A0054
:1080D00025642025642025642025640A004261640B
:1080E000207265636F726420666F756E64206475BC
:1080F00072696E6720696E697469616C697A61740E
:10810000696F6E210A004E6F7420656E6F75676827
:1081100020726F6F6D206576656E20616674657282
:1081200020636F6D70616374696F6E0A00526573CE
:10813000746F72696E67202564207363726970744E
:10814000732E2E2E0053746172746564002D2D2DD4
:108150002D2D0A0050657273697374656E74204D1D
:10816000656D6F727920546573740A0A000A496E4E
:10817000697469616C697A696E67204D656D6F72AB
:10818000790A004D656D6F727920696E7469746942
:10819000616C697A65643B2077726974696E6720E7
:1081A0007265636F7264732E2E2E0A005265636FC0
:1081B0007264206174206F66667365742025643A6A
:1081C000202564202564202564202564202825643A
:1081D00020776F726473290A0046696E616C3A20D9
:1081E00063757272656E74202564207573656420F2
:1081F00025642063302025642063312025640A0033
:10820000E2ECF0F4F8FC00046E756D626572006ECD
:108210006F6E65006F7468657200706169720073DB
:108220007472696E6700726164696F00646973617A
:10823000626C65526164696F006D65737361676537
:108240005265636569766564007061636B6574523D
:10825000656365697665007061636B657453656E0F
:1082600064007265636569766564496E7465676507
:10827000720072656365697665644D6573736167E5
:1082800065547970650072656365697665645374D9
:1082900072696E670073656E64496E7465676572B6
:1082A0000073656E64506169720073656E64537427
:1082B00072696E67007365744368616E6E656C0009
:1082C00073657447726F757000736574506F77656E
:1082D00072007369676E616C537472656E6774685F
:1082E000004E6F2066726565207461736B20656E49
:1082F00074726965730057656C636F6D6520746F88
:10830000204D6963726F426C6F636B7321004D6522
:108310006D6F727920636C65617265642E00416CCB
:108320006C207461736B732073746F70706564007C
:1083300076303534002025732025730007000000B7
:10834000030000006D6963726F3A626974006861CE
:1083500073546F6E6500706C6179546F6E65006860
:108360006173536572766F00736574536572766FCF
:1083700000000000000000000100000002000000FA
:1083800003000000040000000A0000006E65740095
:1083900068617357694669007374617274576946FE
:1083A000690073746F70576946690077696669532D
:1083B0007461747573006D794950416464726573BA
:1083C00073007468696E6744657363726970746979
:1083D0006F6E00636C6561725468696E67446573A3
:1083E0006372697074696F6E00617070656E645459
:1083F0006F5468696E674465736372697074696FFE
:108400006E001A1B1C03040607090A1718191A1B09
:108410001C03040607090A171819646973706C6154
:1084200079006C696768744C6576656C00000000C3
:108430000000000001000000020000000300000036
:108440000400000005000000060000000700000016
:1084500008000000090000000A0000000B000000F6
:108460000C0000000D0000000E0000000F000000D6
:1084700010000000120000001400000016000000B0
:10848000180000001A0000001C0000001E00000080
:10849000200000002300000026000000290000004A
:1084A0002C0000002F000000320000003600000009
:1084B0003A0000003E0000004200000046000000BC
:1084C0004B00000050000000550000005A00000062
:1084D00061000000680000006F00000076000000EE
:1084E0007D000000840000008B000000920000006E
:1084F00099000000A0000000A7000000AE000000EE
:10850000B5000000BC000000C3000000CA0000006D
:10851000D1000000D8000000DF000000E6000000ED
:10852000ED000000F4000000FB000000FF00000070
:10853000000000000008080800080A4A4000000A7D
:108540005FEA5FEA0ED92ED36E19324489330C925A
:108550004C924D08080000000488080804080484B0
:108560008488000A448A4000048EC480000000040D
:108570008800000EC000000000080001224488109E
:108580000C9252524C048C84848E1C824C901E1E81
:10859000C244924C06CA525FE21FF01EC13E024422
:1085A0008ED12E1FE24488100ED12ED12E0ED12E48
:1085B000C48800080008000004800488024488047D
:1085C00082000EC00EC008048244880ED126C0046A
:1085D0000ED135B36C0C925ED2521C925C925C0E42
:1085E000D010100E1C9252525C1ED01C901E1ED039
:1085F0001C90100ED013712E12525ED2521C88089D
:10860000081C1FE242524C12549814921010101081
:108610001E113B75B131113935B3710C9252524C68
:108620001C925C90100C92524C861C925C92510EE3
:10863000D00C825C1FE4848484125252524C11315B
:10864000312A44113135BB7112524C9252112A44D5
:1086500084841EC488101E0EC808080E10080482E8
:10866000410EC242424E048A400000000000001F3A
:108670000804800000000ED2524F10101C925C00C3
:108680000ED0100E02424ED24E0C925C900E06C8D6
:108690001C88080ED24EC24C10101C9252080008C2
:1086A0000808024002424C10149814920808080866
:1086B00006001B75B131001C925252000C92524CB4
:1086C000001C925C90000ED24EC2000ED010100022
:1086D00006C8049808080EC807001252524F00112D
:1086E000312A4400113135BB00124C8C9200112A02
:1086F0004498001EC4881E06C48C84860808080896
:108700000818080C881800000C836073656E736F7E
:1087100072730074656D7065726174757265007452
:10872000696C74580074696C74590074696C745A7B
:1087300000746F75636852656164007466740065E7
:108740006E61626C65446973706C61790073657405
:10875000506978656C006C696E65007265637400C1
:10876000726F756E646564526563740063697263E9
:108770006C6500747269616E676C6500746578740D
:1087800000535049436C6173733A3A535049436CF8
:10879000617373284E52465F5350495F5479706538
:1087A0002A2C2075696E74385F742C2075696E747C
:1087B000385F742C2075696E74385F742900705F9F
:1087C00073706920213D204E554C4C002F55736528
:1087D00072732F6A6F686E6D616C6F6E65792F4C66
:1087E0006962726172792F41726475696E6F313599
:1087F0002F7061636B616765732F73616E6465656C
:10880000706D69737472792F6861726477617265D3
:108810002F6E5246352F302E362E302F6C696272F5
:1088200061726965732F5350492F5350492E6370FD
:108830007000000000000000000000005F49000020
:10884000254900004B4900005549000085490000BA
:108850004949000003000000020000000100000080
:108860000400000005000000110000000C000000E2
:108870000B000000120000000A00000006000000CB
:108880001A0000001400000017000000160000008D
:108890001500000010000000FFFFFFFFFFFFFFFFBB
:1088A000000000001E000000190000001800000079
:1088B0000700000008000000090000000D00000093
:1088C0000E0000000F0000001C0000001B00000054
:1088D0001D000000130000000000000000003043F5
:1088E00000000000000030C3000000000000000095
:1088F00085520000A5510000F55200000953000008
:10890000FF52000083520000775200001553000010
:10891000A1520000735200002C2066756E637469CA
:108920006F6E3A2000617373657274696F6E2022F6
:10893000257322206661696C65643A2066696C65FE
:1089400020222573222C206C696E652025642573F6
:1089500025730A0043000000A0010020232D302BC6
:108960002000686C4C006566674546470030313230
:108970003334353637383941424344454600303187
:1089800032333435363738396162636465660000E6
:1089900020202020202020202028282828282020AF
:1089A00020202020202020202020202020202020C7
:1089B000881010101010101010101010101010103F
:1089C000040404040404040404041010101010101F
:1089D00010414141414141010101010101010101F8
:1089E000010101010101010101010110101010102C
:1089F00010424242424242020202020202020202C9
:108A000002020202020202020202021010101020F0
:108A10000000000000000000000000000000000056
:108A20000000000000000000000000000000000046
:108A30000000000000000000000000000000000036
:108A40000000000000000000000000000000000026
:108A50000000000000000000000000000000000016
:108A60000000000000000000000000000000000006
:108A700000000000000000000000000000000000F6
:108A800000000000000000000000000000000000E6
:108A900000000000000000000000000000000000D6
:108AA00000000000000000000000000000000000C6
:108AB00000000000000000000000000000000000B6
:108AC00000000000000000000000000000000000A6
:108AD0000000000000000000000000000000000096
:108AE0000000000000000000000000000000000086
:048AF0000000000082
:088AF4008076FF7F0100000005
:108AFC00FFFFFFFF2C820000E926000039820000F6
:108B0C00012A000049820000A129000057820000C0
:108B1C008D2B00006282000005270000728200008D
:108B2C006D2700008682000015270000958200004A
:108B3C00A72C0000A1820000312C0000AA820000AA
:108B4C00D72B0000B58200001D290000C082000058
:108B5C00A5280000C9820000D9280000D28200009C
:108B6C001D27000019FCFFFFFFFFFFFF4E830000D5
:108B7C002539000056830000213900005F83000076
:108B8C0029390000688300002D3900009083000013
:108B9C00DD3B000098830000013C0000A283000034
:108BAC000B3C0000AB830000153C0000B6830000BA
:108BBC001F3C0000C2830000EB3B0000D38300008D
:108BCC00F53B0000E9830000E13B0000228400003B
:108BDC00413C000018000000FF000000138700005B
:108BEC00514400001F870000194700002587000032
:108BFC00294700002B87000039470000318700000F
:108C0C00854400003F870000514700004D8700005D
:108C1C005547000056870000594700005B8700004D
:108C2C005D47000060870000614700006C87000012
:108C3C0065470000738700004D4700007C870000EB
:108C4C00494700000300000002000000080000007B
:108C5C000A000000FFFFFFFF000000000100000001
:108C6C000000020001000000FFFFFFFF00000000F9
:108C7C00020000000000040002000000FFFFFFFFE4
:108C8C0000000000030000000000080003000000CA
:108C9C0000000000908A0000B08A0000D08A00001A
:108CAC0000000000000000000000000000000000B8
:108CBC0054890000000000000000000000000000CB
:108CCC000000000000000000000000000000000098
:108CDC000000000000000000000000000000000088
:108CEC000000000000000000000000000000000078
:108CFC00A00100208F89000039010000F548000018
:108D0C00D94B0000795500000D0100000000000057
:0400000300004D3577
:00000001FF
